:100000000C9463000C948B000C948B000C948B006C
:100010000C948B000C948B210C948B000C948B0013
:100020000C948B000C948B000C948B000C948B0024
:100030000C948B000C948B000C948B000C948B0014
:100040000C9422200C948B000C94F01F0C94CA1F6B
:100050000C948B000C948B000C948B000C948B00F4
:100060000C946C200C948B000000000024002700EE
:100070002A000000000023002600290000000000E4
:10008000250028002B0004040404040404040202D4
:100090000202020203030303030301020408102007
:1000A0004080010204081020010204081020000012
:1000B0000008000201000003040700000000000027
:1000C0000000EF210E3111241FBECFEFD8E0DEBFBC
:1000D000CDBF27E0A0EEB4E001C01D92A135B2076C
:1000E000E1F714E0A0E0B1E0ECEEF0E702C005902B
:1000F0000D92A03EB107D9F710E0C2E6D0E004C0EF
:100100002197FE010E945A36C136D107C9F70E94D5
:1001100022230C9469380C9400002091EB0581E0B7
:10012000213208F044C08091C7058111FCCF809135
:10013000EA0592E09093C70591E09093C6059FEF82
:100140009093C5051092C4052093C305AAECB5E0B1
:10015000E3EAF5E090E0291331C01092A2059091F6
:10016000A205880F892B8093A2058091A10581307B
:1001700049F51092A1058091A2058093BB00809162
:10018000BC0083FDF8CF85EC8093BC008091C7054F
:100190008230E1F38091C5058F3FB1F08091C505B4
:1001A0008032A1F08091C505803391F084E01092F7
:1001B000C9051092EB051092C80508953D91319341
:1001C0009F5FC9CF85EEE0CF80E0F1CF82E0EFCF37
:1001D00083E0EDCF9B01AC01E091FC05F091FD05C2
:1001E00082E08083211581EE380741055105E9F150
:1001F00060E079E08DE390E00E9493342150310972
:10020000410951095695479537952795E091F8058D
:10021000F091F9051082E091FA05F091FB05208339
:1002200010920406E0910006F091010686E08083BA
:10023000E091FE05F091FF05808180618083E0916F
:10024000FE05F091FF05808188608083E091FE05C6
:10025000F091FF05808180688083E091FE05F09138
:10026000FF0580818F7D80830895E091FC05F091EA
:10027000FD05108220E1CACF80917F059091800515
:10028000891B990B08952F923F924F925F926F9224
:100290007F928F929F92AF92BF92CF92DF92EF9216
:1002A000FF920F931F93CF93DF93CDB7DEB76C9779
:1002B0000FB6F894DEBF0FBECDBF522E3D874E87DE
:1002C000252E462E372E782E692EA982BF86C88A03
:1002D000D98AEA8AFB8A0C8B1D8B988E8F8A21150E
:1002E00000EA30070CEA400709EB500703E060071B
:1002F00071058105910509F098F52F3F10EE310742
:1003000015EF410715E0510761057105810591055C
:1003100009F008F40BC12F3F354D41415E47634062
:1003200071058105910509F008F40BC129813F850C
:10033000488959896A897B898C899D89A0E099249B
:1003400093940E944E36C9F4F1E0FE8B04E0802EB7
:10035000912CA12CB12C89869A86AB86BC8616C1BD
:10036000512CB0EABD87ECEAEE8789EB282E93E0AA
:10037000492E312C712C612CD9CFA52CBD84CE8473
:10038000D22CE42CF32C072D162D29813F8548898A
:1003900059896A897B898C899D890E949935298729
:1003A0003A874B875C8729853A854B855C85B6E023
:1003B000AB2EB12C263031054105510568F08985F9
:1003C0009A85AB85BC8589309740A105B105E0F0E1
:1003D000F8E0AF2EA7E0BA2EC12CD12CE12CF12CE5
:1003E00000E010E029813F85488959896A897B8925
:1003F0008C899D890E949935522E3D874E87252EE6
:10040000462E372E782E692EA52CBD84CE84D22C74
:10041000E42CF32C072D162D29813F854889598915
:100420006A897B898C899D890E949735AA24AA9420
:10043000BB24BA94EFE0CE2ED12CE12CF12C00E0BD
:1004400010E00E94D434A52CBD84CE84D22CE42CA0
:10045000F32C072D162D0E949935A32FF42FE52F8D
:10046000422F5A2F6F2F7E2FCC24CA94DC2C8FE082
:10047000E82EF12C411551056105710521F4C12CBF
:10048000D12C7601C394AA24A3949A1409F4E5C04C
:1004900001E00E8BCB01BA0137E0660F771F881F92
:1004A000991F3A95D1F7A70196010E949334298F9D
:1004B0003A8F4B8F5C8F89849A84AB84BC8447E0ED
:1004C000880C991CAA1CBB1C4A95D1F79501840184
:1004D00012502109310948015901298D3A8D4B8D5E
:1004E0005C8D280D391D4A1D5B1DAF89B88D2D937C
:1004F0003D934D935C931397FD01648375838683CD
:1005000097831896CD92DD92ED92FC921B978E8880
:10051000882009F481C059829D849F86AE84A88A70
:10052000298A4A8A3B8A7C8A6D8A76C0512C01EEE0
:100530000D8715EF1E8725E0222E412C312C712CC2
:10054000612C29813F85488959896A897B898C89F1
:100550009D89A0E0912C0E944E3609F00ECFA52C6B
:10056000BD84CE84D22CE42CF32C072D162D20E054
:1005700034E04BE654EF64E170E080E090E00E94EC
:10058000993529873A874B875C871E8A89849A84A4
:10059000AB84BC84A501940160E070E0CB01A52C84
:1005A000BD84CE84D22CE42CF32C072D162D298368
:1005B0003A834B835C836D837E838F83988760E06F
:1005C00070E080E090E00E94D43429833F87488B1C
:1005D000598B6A8B7B8B8C8B9D8B0E89C12CD12C7C
:1005E0007601C39440E050E0BA01013009F052CFE7
:1005F000AF89B88D1D921D921D921C921397FD011B
:10060000148215821682178281E090E0A0E0B0E0AB
:1006100080879187A287B38729813F854889598937
:100620006A897B898C899D896C960FB6F894DEBFA8
:100630000FBECDBFDF91CF911F910F91FF90EF9033
:10064000DF90CF90BF90AF909F908F907F906F90F2
:100650005F904F903F902F900895AF89B88D1D9275
:100660001D921D921C921397FD0114821582168211
:10067000178281E090E0A0E0B0E080879187A287B8
:10068000B3875982FD85FF878E84888A49CFDF92A0
:10069000EF92FF920F931F93CF93DF93FC01E080C3
:1006A000F18002811381D481C581B681D780970101
:1006B000A8016D2F7C2F8B2F9D2D35534C40510958
:1006C00061097109810991092F3F34434C4051055B
:1006D000610571058105910509F0D0F49701A80124
:1006E0006D2F7C2F8B2F9D2D07E00E9406362083D7
:1006F000318342835383648375838683978387E042
:10070000DF91CF911F910F91FF90EF90DF900895AF
:100710009701A8016D2F7C2F8B2F9D2D3A564841B4
:10072000510961097109810991092F3F39464841F1
:100730005105610571058105910509F098F497014E
:10074000A8016D2F7C2F8B2F9D2D06E00E94063671
:1007500020833183428353836483758386839783A5
:1007600086E0CECF9701A8016D2F7C2F8B2F9D2D7A
:10077000345D4043510961097109810991092F3F95
:10078000334D40435105610571058105910509F01F
:1007900098F49701A8016D2F7C2F8B2F9D2D05E0DC
:1007A0000E9406362083318342835383648375839A
:1007B0008683978385E0A4CF9701A8016D2F7C2FB6
:1007C0008B2F9D2D385A41465109610971098109C4
:1007D00091092F3F374A4146510561057105810551
:1007E000910509F098F49701A8016D2F7C2F8B2FAC
:1007F0009D2D04E00E94063620833183428353837B
:10080000648375838683978384E07ACF9701A801F8
:100810006D2F7C2F8B2F9D2D3055434C5109610935
:100820007109810991092F3F3F44434C51056105EE
:1008300071058105910509F098F49701A8016D2FC4
:100840007C2F8B2F9D2D03E00E9406362083318361
:1008500042835383648375838683978383E050CF79
:100860009701A8016D2F7C2F8B2F9D2D305A464864
:10087000514061097109810991092F3F3F4946485B
:100880005140610571058105910509F098F49701C2
:10089000A8016D2F7C2F8B2F9D2D02E00E94063624
:1008A0002083318342835383648375838683978354
:1008B00082E026CF9701A8016D2F7C2F8B2F9D2DD5
:1008C00030544D40534061097109810991092F3F0E
:1008D0003F434D405340610571058105910509F085
:1008E00098F49701A8016D2F7C2F8B2F9D2D01E08F
:1008F0000E94063620833183428353836483758349
:100900008683978381E0FCCE80E0FACE0895089537
:100910000895DB0114964D915C9115976D917C9132
:10092000DC01ED91FC910280F381E02D0994AF92FE
:10093000BF92CF92DF92EF92FF920F931F93CF93CC
:10094000DF936C017B018B01040F151FEB015E012E
:10095000AE18BF08C017D10759F06991D601ED91C3
:10096000FC910190F081E02DC6010995892B79F762
:10097000C501DF91CF911F910F91FF90EF90DF9014
:10098000CF90BF90AF900895FC01538D448D252FDB
:1009900030E0842F90E0821B930B541710F0CF9619
:1009A000089501970895FC01918D828D981761F04B
:1009B000A28DAE0FBF2FB11D5D968C91928D9F5F62
:1009C0009F73928F90E008958FEF9FEF0895FC0141
:1009D000918D828D981731F0828DE80FF11D858DF4
:1009E00090E008958FEF9FEF0895FC01918D228D87
:1009F000892F90E0805C9F4F821B91098F7399270C
:100A000008958CEE95E00E94F50421E0892B09F40D
:100A100020E0822F089580E090E0892B29F00E9449
:100A2000010581110C9400000895FC01A48DA80F0C
:100A3000B92FB11DA35ABF4F2C91848D90E0019620
:100A40008F739927848FA689B7892C93A089B18940
:100A50008C91837080648C93938D848D981306C0E1
:100A60000288F389E02D80818F7D80830895EF9245
:100A7000FF920F931F93CF93DF93EC0181E0888F58
:100A80009B8D8C8D98131AC0E889F989808185FF28
:100A900015C09FB7F894EE89FF896083E889F989CA
:100AA00080818370806480839FBF81E090E0DF91CC
:100AB000CF911F910F91FF90EF900895F62E0B8D1F
:100AC00010E00F5F1F4F0F731127E02E8C8D8E11DA
:100AD0000CC00FB607FCFACFE889F989808185FF41
:100AE000F5CFCE010E941505F1CFEB8DEC0FFD2F58
:100AF000F11DE35AFF4FF0829FB7F8940B8FEA89FC
:100B0000FB8980818062CFCFCF93DF93EC01888D0A
:100B10008823B9F0AA89BB89E889F9898C9185FD78
:100B200003C0808186FD0DC00FB607FCF7CF8C9106
:100B300085FFF2CF808185FFEDCFCE010E941505A4
:100B4000E9CFDF91CF910895833081F028F481308F
:100B500099F08230A9F008958730A9F08830C9F063
:100B60008430B1F4809180008F7D03C0809180003B
:100B70008F7780938000089584B58F7784BD089522
:100B800084B58F7DFBCF8091B0008F778093B000CC
:100B900008958091B0008F7DF9CFCF93DF93282FF8
:100BA00030E0F901E255FF4F8491F901E656FF4F1D
:100BB000D491F901EA57FF4FC491CC2389F08111F8
:100BC0000E94A405EC2FF0E0EE0FFF1FE458FF4F4A
:100BD000A591B4918FB7F894EC91DE2BDC938FBF85
:100BE000DF91CF9108951092800510927F051092A9
:100BF000C9051092EB051092C70581E08093C605E8
:100C00001092A10582E10E94CD0583E10E94CD05ED
:100C1000E9EBF0E080818E7F808380818D7F80830F
:100C200088E48093B80085E48093BC0086E894E073
:100C300090937E0580937D0587E894E090937C05F2
:100C400080937B050895CF93DF93282F30E0F9013F
:100C5000E255FF4F8491F901E656FF4FD491F90117
:100C6000EA57FF4FC491CC23A1F081110E94A40543
:100C7000EC2FF0E0EE0FFF1FEE58FF4FA591B4915F
:100C8000EC91ED2381E090E009F480E0DF91CF91D9
:100C9000089580E090E0FACFCF93DF9390E0FC01DD
:100CA000E656FF4F24918A579F4FFC018491882379
:100CB000C9F090E0880F991FFC01E859FF4FA591FA
:100CC000B491FC01E458FF4FC591D49161110DC05E
:100CD0009FB7F8948C91209582238C938881282348
:100CE00028839FBFDF91CF910895623051F49FB761
:100CF000F8943C91822F809583238C93E8812E2B4E
:100D0000EFCF8FB7F894EC912E2B2C938FBFEACFB7
:100D10008E3008F08E508770806480937C008091C4
:100D20007A00806480937A0080917A0086FDFCCFFF
:100D3000809178009091790008953FB7F894809160
:100D4000340590913505A0913605B091370526B54B
:100D5000A89B05C02F3F19F00196A11DB11D3FBFF3
:100D6000BA2FA92F982F8827BC01CD01620F711DC2
:100D7000811D911D42E0660F771F881F991F4A95BC
:100D8000D1F708958F929F92AF92BF92CF92DF9248
:100D9000EF92FF926B017C010E949D064B015C016A
:100DA000C114D104E104F104B9F00E949D06681950
:100DB00079098A099B09683E73408105910580F392
:100DC00021E0C21AD108E108F10888EE880E83E01C
:100DD000981EA11CB11CE4CFFF90EF90DF90CF9044
:100DE000BF90AF909F908F90089585ED8093BC0049
:100DF0008091BC0084FDFCCF1092C705089520911E
:100E00001005260F3327331F21323105ECF42091D2
:100E1000C705FC0190E080E0243069F082E008958D
:100E2000A09110052191AC0140515B4FA40FB52F4B
:100E3000B11D2C930196861798F380911005680FC9
:100E40006093100580E0089581E008950895E09191
:100E5000800580917F05E81730F4F0E0EF57FA4FF6
:100E6000808190E008958FEF9FEF08959091800525
:100E700080917F052FEF3FEF981748F4E92FF0E0BE
:100E8000EF57FA4F208130E09F5F90938005C901B2
:100E90000895CF92DF92EF92FF920F931F93CF931B
:100EA000DF937C01CB018A012091C805222389F0C0
:100EB000EB016B01C40ED51ECC15DD0569F06991FF
:100EC000D701ED91FC910190F081E02DC7010995CA
:100ED000F3CF642F0E94FF06C801DF91CF911F91CD
:100EE0000F91FF90EF90DF90CF900895CF93DF9315
:100EF0001F92CDB7DEB769832091C8052223F9F090
:100F00002091EB05203258F021E030E0FC013383E2
:100F1000228390E080E00F90DF91CF91089580913F
:100F2000C905E82FF0E0E653FA4F998190838F5F6F
:100F30008093C9058093EB0581E090E0ECCF61E000
:100F4000CE0101960E94FF06F7CFCF93C62F91E006
:100F50009093C80590E69093EA051092C905109207
:100F6000EB05682F89E896E00E9476076C2F89E8E8
:100F700096E00E947607CF910C948D000F931F93FB
:100F8000CF93DF938B0191E09093C80590E6909307
:100F9000EA051092C9051092EB05682F89E896E0E2
:100FA0000E947607E801085F1F4F699189E896E083
:100FB0000E947607C017D107C1F7DF91CF911F912B
:100FC0000F910C948D00FC01248131E03093C80511
:100FD0002093EA051092C9051092EB058385682BD2
:100FE00089E896E00E9476070C948D0090E080E0FE
:100FF000089580913901813091F480E096E9A0E074
:10100000B0E08093450190934601A0934701B093CF
:10101000480160E076E980E090E00E94EA0080917B
:101020003901823091F480E091EEA0E0B0E080934D
:10103000450190934601A0934701B093480160E0B9
:1010400071EE80E090E00E94EA00809139018330E7
:1010500091F480E092ECA1E0B0E0809345019093A0
:101060004601A0934701B093480160E072EC81E033
:1010700090E00C94EA0008958091760590917705B0
:10108000029799F480913A01833078F084E690E0F9
:10109000A0E0B0E080935C0190935D01A0935E01BD
:1010A000B0935F0183E080933A0180913A0190917F
:1010B000EE048917C9F08130C1F481E090E0A0E02E
:1010C000B0E080935C0190935D01A0935E01B093CA
:1010D0005F0180913A01811103C081E080933A0160
:1010E00080913A018093EE040895823029F48AE0D9
:1010F00090E0A0E0B0E0E5CF833029F484E690E012
:10110000A0E0B0E0DECF843029F488EE93E0A0E0E8
:10111000B0E0D7CF853029F480E197E2A0E0B0E0DD
:10112000D0CF863029F480EA96E8A1E0B0E0C9CFBC
:10113000873029F480E492E4AFE0B0E0C2CF883099
:1011400040F287E080933A01C4CF8091440181113D
:1011500004C081E0809366050895833011F486E22F
:10116000F9CF843011F482E3F5CF853011F48FE3A9
:10117000F1CF8630C1F3873011F488E5EBCF8830AA
:1011800011F484E6E7CF893011F48EE4E3CF8A309E
:1011900019F781E7DFCFCF93DF9391E09093C805F4
:1011A00090E69093EA051092C9051092EB05682F1E
:1011B00089E896E00E9476070E948D008091C7051D
:1011C0008111FCCF81E08093C7051092C6059FEF87
:1011D0009093C5051092C4051092C3058093A20593
:1011E0008091A205806C8093A2058091A105813039
:1011F00061F51092A1058091A2058093BB008091BA
:10120000BC0083FDF8CF85EC8093BC008091C705BE
:101210008130E1F38091C405811119C08091C4052A
:10122000E3EAF5E0A1E8B5E0C0E0C81312C010920F
:101230008005C0937F0580918005C81771F089E80B
:1012400096E00E943607D82FF6CF85EEDDCF81E0FD
:10125000E7CF91919D93CF5FE8CF8D2FDF91CF9115
:101260000895CF93DF93D82FC62F83E00E94CB0839
:1012700061E070E001C0660FDA95EAF7C13039F439
:101280006095682383E0DF91CF910C94A507682BCC
:10129000F9CF0F931F93CF938B01C0E1C80F8C2F11
:1012A0000E94CB08682F012B39F46F7D8C2FCF91D2
:1012B0001F910F910C94A5076062F8CF0F931F93B5
:1012C000CF938C01C62F0E94E3076C2F6460C80186
:1012D0000E94E3076C2F6B7FC8010E94E30783EC39
:1012E00090E00197F1F7CF911F910F9108950F931F
:1012F0001F93CF93DF938C01D62FC42F607F642B75
:101300000E945E0980E1D89FB00111246C2BC801B6
:10131000DF91CF911F910F910C945E09CF93DF93D2
:10132000CDB7DEB728970FB6F894DEBF0FBECDBF9E
:1013300098E0E2E7F1E0DE01119601900D929A95B6
:10134000E1F790914907961708F46FEF262F30E0E8
:10135000220F331F41E050E04C0F5D1F240F351F5B
:10136000F9016081680F606840E081E497E02896A9
:101370000FB6F894DEBF0FBECDBFDF91CF910C94B6
:10138000770941E00E94770981E090E0089541E00B
:10139000682F81E497E00E94770981E090E008954A
:1013A00040E061E081E497E00E9477098BE39FE1F0
:1013B0000197F1F708950F931F93CF93DF938B015C
:1013C00098E0899FB0011124606440E081E497E0D7
:1013D0000E947709E801085F1F4F699181E497E057
:1013E0000E94C109C017D107C1F7DF91CF911F91AA
:1013F0000F910895FB0101900020E9F73197AF01AB
:10140000461B570BDC01ED91FC910280F381E02D2E
:1014100009948F929F92AF92BF920F931F93CF9395
:10142000DF93CDB7DEB7A1970FB6F894DEBF0FBE3E
:10143000CDBF19A2423008F44AE08E010F5D1F4F64
:10144000842E912CB12CA12CA50194010E949334DF
:10145000E62FB901CA01EA3004F5E05DD801EE9348
:101460008D01232B242B252B79F790E080E010971A
:1014700029F0BD0181E497E00E94FA09A1960FB618
:10148000F894DEBF0FBECDBFDF91CF911F910F91BA
:10149000BF90AF909F908F900895E95CDFCFCF927F
:1014A000DF92EF92FF92CF93DF9397FF19C06B010A
:1014B0007C018DE20E94C709EC0166277727CB01EA
:1014C0006C197D098E099F094AE00E94090A8C0F58
:1014D0009D1FDF91CF91FF90EF90DF90CF90089507
:1014E0004AE0DF91CF91FF90EF90DF90CF900C9486
:1014F000090ACF92DF92EF92FF92C0904B05D090F5
:101500004C05E0904D05F0904E058AE0C816D104D8
:10151000E104F1041CF480E20E94C70980E20E9409
:10152000C709C701B6010E944F0A8EE20E94C7098F
:1015300060914F0570915005809151059091520531
:1015400020E432E44FE050E00E94B53428EE33E06E
:1015500040E050E00E94B53469017A01C0924B0529
:10156000D0924C05E0924D05F0924E0584E6C816E7
:10157000D104E104F10464F480E30E94C7098AE025
:10158000C816D104E104F1041CF480E30E94C709E9
:10159000C701B6010E944F0A8EE20E94C7096091FE
:1015A0004F0570915005809151059091520528EE9C
:1015B00033E040E050E00E94B5346B017C01C09202
:1015C0004B05D0924C05E0924D05F0924E0584E615
:1015D000C816D104E104F10464F480E30E94C70951
:1015E0008AE0C816D104E104F1041CF480E30E94EF
:1015F000C709C701B601FF90EF90DF90CF900C9420
:101600004F0A4F925F926F927F928F929F92AF920A
:10161000BF92CF92DF92EF92FF920F931F93CF93DF
:101620006B017C01742EAC019B010E948E3466EC30
:1016300071E0811126C046015701E894B7F82FEFF9
:101640003FEF4FE75FE7C501B4010E948E3481117F
:101650000CC02FEF3FEF4FE75FE7C501B4010E94D9
:10166000F4316AEC71E0181664F02FEF3FEF4FE7AA
:101670005FE4C701B6010E9489341816ACF46EEC21
:1016800071E081E497E0CF911F910F91FF90EF906F
:10169000DF90CF90BF90AF909F908F907F906F9092
:1016A0005F904F900C94FA092FEF3FEF4FE75FECFC
:1016B000C701B6010E94F43187FDE1CF20E030E0A0
:1016C000A901C701B6010E94F43110E000E087FFD4
:1016D00008C08DE20E94C7098C01F7FAF094F7F870
:1016E000F094C0E060E070E080E09FE37C1641F0A1
:1016F00020E030E040E251E40E94E133CF5FF6CFDA
:10170000A70196010E9475332B013C010E945A34B7
:101710004B015C014AE00E94090A7C01E00EF11EC7
:10172000CC23B1F1C501B4010E94F9319B01AC0198
:10173000C301B2010E9474334B015C018EE20E942E
:10174000C709E80EF91EC15018F120E030E040E270
:1017500051E4C501B4010E945A322B013C010E94A0
:101760005A344B01B12CA12C4AE0C501B4010E94AE
:10177000090AE80EF91EC501B4010E94F9319B0166
:10178000AC01C301B2010E9474334B015C01DBCF99
:10179000C701CF911F910F91FF90EF90DF90CF90F5
:1017A000BF90AF909F908F907F906F905F904F9081
:1017B00008950C94FA0960E083E00E948E0960911C
:1017C0006F0570917005809171059091720560931D
:1017D0004F0570935005809351059093520520E476
:1017E00032E44FE050E00E94B53420934B05309333
:1017F0004C0540934D0550934E050E94790A64E6CE
:1018000073E081E497E00C94D90B2F923F924F92B2
:101810005F926F927F928F929F92AF92BF92CF9280
:10182000DF92EF92FF920F931F93CF93DF93CDB789
:10183000DEB76A970FB6F894DEBF0FBECDBF2F8B11
:101840003987488F598F6A877A8F1C011E8B0D8BC1
:1018500060913D0770913E0780913F07909140074E
:1018600024E630E040E050E00E943B35522E632EEB
:10187000742E852E962E788B8F87492E8091370770
:1018800090913807A0913907B0913A076C017D011A
:10189000FF0CCC08DC2C76019C01AD016C2D7C2D5D
:1018A0008C2D9C2D0FE10E940636A12CEAECBE2E59
:1018B000FAE9CF2EABE3DA2EE12CF12C00E010E0B8
:1018C0000E946835A52CB62CC72CD82CE92CF8889A
:1018D0000F85142D0E94D4340FE10E9421362983F4
:1018E0003A834B835C836D837E838F839887898162
:1018F0009A81AB81BC81BB0F880B982FDC018B8751
:101900009C87AD87BE87252D362D472D582D692DF7
:101910007F2D8F85942DA980BA80CB80DC80EB84CD
:10192000FE2C0E2D1E2D0E943C3629833B874F87AF
:10193000588B698B7A8B8B8B9C8B8F889A8C282DFC
:101940003985488D598D6A85792DC101211534401D
:101950004B46544F644171058105910569F060F073
:10196000812CB4E0B987EBE6E88FF4EFF98F84E1DE
:101970008A87912C212C312C282D3985488D598D21
:101980006A85792DC101211538454744584F6D406E
:1019900071058105910560F4812CB8E5B987E7E40C
:1019A000E88FF8EFF98F8DE08A87912C212C312C6C
:1019B000A980BB84CF84D888E988FA880B891C89E0
:1019C000282D3985488D598D6A85792DC1010E9450
:1019D000993529013A011FE0A12E9FE049165104D3
:1019E0006104710440F0ABE54A16510461047104CE
:1019F000D0F0BAE5AB2EB12CC12CD12CE12CF12CBE
:101A000000E010E029813B854F85588969897A89F2
:101A10008B899C890E94D434822E3987488F598FB4
:101A20006A87972E1C01A980BB84CF84D888E98857
:101A3000FA880B891C89282D3985488D598D6A852E
:101A4000792DC1010E949735AA24AA94BB24BA9487
:101A5000AFE0CA2ED12CE12CF12C00E010E00E9466
:101A6000D434A980BB84CF84D888E988FA880B89CC
:101A70001C890E949935C901DA01812C912C5401ED
:101A800083940097A105B10531F088248A94982C9D
:101A9000EFE0AE2EB12CBC01CD0127E0660F771F21
:101AA000881F991F2A95D1F7A50194010E949334AC
:101AB000362E272E182F67E0440C551C661C771C09
:101AC0006A95D1F7B2E05B1A61087108420E531EA5
:101AD000641E751E84E190E00E9460369A838983BB
:101AE000FC0190828182862D83708283538244829E
:101AF0007CE0B694A794979487947A95D1F7F82DC3
:101B0000F07F8F2E812AA981BA8115968C92159724
:101B100016962C92169717963C921797ED89FE8988
:101B2000BD018AE1EF2B19F069817A8182E20E947E
:101B3000BE0789819A816A960FB6F894DEBF0FBE00
:101B4000CDBFDF91CF911F910F91FF90EF90DF906C
:101B5000CF90BF90AF909F908F907F906F905F904D
:101B60004F903F902F900C94FC362F923F924F92C3
:101B70005F926F927F928F929F92AF92BF92CF921D
:101B8000DF92EF92FF920F931F93CF93DF93CDB726
:101B9000DEB72D970FB6F894DEBF0FBECDBF3C0168
:101BA000C982DA82EB82FC820D831E832F83388701
:101BB00049875A876B877C878AA18D873C2C2D2C7F
:101BC0009E2C502E412EB22EC984DA84EB84FC84E4
:101BD00084E190E00E9460368C01FC01D082C182D9
:101BE000862D880F880F880F845D0E94CB08F92D01
:101BF000F3709F2E8C7F982AF80192822382348280
:101C00004CE0F694E794D794C7944A95D1F7FC2D0D
:101C1000F07FCF2E8B2D8F70C82AF801C5824682A7
:101C20005782B80182E3F1E06F16710431F082E06F
:101C30006816710409F447C08AE20E94BE0730E1C9
:101C4000F32EF60C8F2D0E94CB0891E0682FA9127D
:101C50003CC060648F2D0E94A507E1E06E16710400
:101C6000B1F1F2E06F167104B9F1A09234072CE2E1
:101C7000F22E8F2D0E94CB0883789D8591118C6068
:101C8000E0E18E9EB0011124682B8F2D0E94A507E4
:101C9000C8012D960FB6F894DEBF0FBECDBFDF9101
:101CA000CF911F910F91FF90EF90DF90CF90BF9059
:101CB000AF909F908F907F906F905F904F903F90EC
:101CC0002F900C94FC368AE3B8CF6F7BC3CFA092E1
:101CD000350794E3F92ECDCFA09236078CE3F82E8A
:101CE000C8CF2F923F924F925F926F927F928F92C6
:101CF0009F92AF92BF92CF92DF92EF92FF920F939B
:101D00001F93CF93DF93CDB7DEB7AC970FB6F894A0
:101D1000DEBF0FBECDBF298F3A8F4B8F5C8F6D8F8B
:101D20007E8F8F8F98A3AAA2BBA216012701702EC7
:101D3000612E9CA68BA69501A601B701802F912F3D
:101D4000A0E00E944E3691F038554744584F6D4000
:101D500071098109910921153C4A43425C4F664053
:101D600071058105910511F008F0C7C1298D3A8DE3
:101D70004B8D5C8D6D8D7E8D8F8D98A12F3F344363
:101D80004C405105610571058105910509F050F43C
:101D9000198E85E38A8F8CE08B8F1C8E1D8E1E8E94
:101DA0001F8E18A2298D3A8D4B8D5C8D6D8D7E8D89
:101DB0008F8D98A12115304A4C4A594B63407105CB
:101DC0008105910569F060F0198E80EA8A8F8CEAAE
:101DD0008B8F89EB8C8F83E08D8F1E8E1F8E18A2C8
:101DE000CE0149960E9447038AA72AA13BA1A101DF
:101DF000B201872D962DA0E0B98DFA8DEB8D0E9452
:101E00004E3609F496C0AC8D1D8D19A38E8D8EA310
:101E10009F8D9FA318A118A72B2F3F2F4E2F5A2F0E
:101E200069A1782F892F912F2F3F15ED310711E1EF
:101E300041071EE7510713E0610771058105910510
:101E400011F008F076C0CE010D964C01AAA0BBA0FF
:101E500061017201072D162D8FA198A50E944301E3
:101E6000798D6A8D5B8D4C8D3D8D2E8D9F8D88A1DA
:101E7000EBA5FCA5E130F105D1F1329709F448C09A
:101E800070931C0760931D0750931E0740931F0714
:101E900030932007209321079093220780932307F4
:101EA00019A619A2F9A5FF938AA4A9A4CD84DE845A
:101EB000EF84F88809891A892B893C894D895E89C4
:101EC0006F89788D8BA59CA50E94B50D0F9019A1E7
:101ED000113009F052C20CA11DA12AA13BA1A10100
:101EE000B201872D962D0E94050C19A246C270934F
:101EF00024076093250750932607409327073093C4
:101F000028072093290790932A0780932B07C8CF8F
:101F100070932C0760932D0750932E0740932F0743
:101F20003093300720933107909332078093330723
:101F3000B7CF1C8D19A38D8D9E8D1F8D1FA3A8A1BA
:101F40002B2F3F2F4E2F59A1BC01812F9A2F2F3FAE
:101F500015ED310711E141071EE7510713E0610755
:101F600071058105910509F008F47CC0CE010D963C
:101F70004C01A12CB12CC12CD12CE12CF12C00E076
:101F800010E08FA19A2F0E9443012AA33BA31A01BC
:101F90002B01782E692E91E099A7E98DECA3FA8D9B
:101FA000FEA3EB8DEFA3FC8DF8A7BD8DAE8DFF8D4D
:101FB000E8A18BA59CA58130910509F455C0029735
:101FC00009F490C1CE010D964C01A12CB12CC12C6D
:101FD000D12CE12CF12C00E010E02CA13EA14FA16E
:101FE00058A56B2F7A2F8F2F9E2F0E9443012AA373
:101FF0003BA31A012B01782E692E70E060E090E07F
:1020000080E00E9449099AA190930C07EBA1E0930C
:102010000D0720920E0730920F0740921007509242
:1020200011077092120760921307898D80931C0725
:102030008A8D80931D078B8D80931E078C8D8093D6
:102040001F078D8D809320078E8D809321078F8DA4
:102050008093220788A180932307F1E0F9A31DA2B2
:102060001CA220CF19A699CF80913C07823009F09D
:10207000FFC02CA13EA14FA158A56B2F7A2F8F2F07
:102080009E2F30584A4156406109710981099109D2
:102090002F37304E424758496240710581059105FE
:1020A00079F170F120912C0730912D0740912E0786
:1020B00050912F076091300770913107809132075E
:1020C00090913307ACA0BEA0CFA0D8A4EB2EFA2EDF
:1020D0000F2F1E2F0E94453699F010922407109260
:1020E00025071092260710922707109228071092B2
:1020F000290710922A0710922B0781E089A33DC17E
:10210000909114079AA3109115071BA3209016070E
:1021100030901707409018075090190770901A07D1
:1021200060901B07CE010D964C01AAA0B12E610153
:102130007201072D162D2CA13EA14FA158A56B2F82
:102140007A2F8F2F9E2F0E94430161E070E081E083
:1021500090E00E94490919A2298D3A8D4B8D5C8D22
:102160006D8D7E8D8F8D98A130584A415640610902
:102170007109810991092F37304E42475849624011
:1021800071058105910509F008F4A8C081E08093EC
:102190003C0720912C0730912D0740912E0750913C
:1021A0002F0760913007709131078091320790912D
:1021B0003307A0E00E944E36F1F18CE297E00E94D6
:1021C00047038AA7A0901407B0901507C090160780
:1021D000D0901707E0901807F090190700911A07A0
:1021E00010911B0720912C0730912D0740912E074D
:1021F00050912F076091300770913107CE01019601
:102200004C0180913207909133070E9443011F9245
:102210008AA4A12CC980DA80EB80FC800D811E810C
:102220002F81388549855A856B857C8582E090E0D1
:102230000E94B50D0F90898D809324078A8D80931D
:1022400025078B8D809326078C8D809327078D8D96
:10225000809328078E8D809329078F8D80932A077E
:1022600088A180932B07E1E0F0E0FDA3ECA31ACE58
:102270009AA1909314071BA110931507209216079B
:1022800030921707409218075092190770921A0758
:1022900060921B07CE010D964C01A12CB12CC12CD4
:1022A000D12CE12CF12C00E010E02CA13EA14FA19B
:1022B00058A56B2F7A2F8F2F9E2F0E9443012AA3A0
:1022C0003BA31A012B01782E692E61E070E081E0BA
:1022D00090E00E94490991E099A33ECF88E0809365
:1022E0003C07A9CF10913C0719A3113009F013C185
:1022F0002CA13EA14FA158A56B2F7A2F8F2F9E2F77
:1023000030584A41564061097109810991092F37B6
:10231000304E42475849624071058105910509F0E8
:1023200008F445C020912C0730912D0740912E07CD
:1023300050912F07609130077091310780913207DB
:1023400090913307ACA0BEA0CFA0D8A4EB2EFA2E5C
:102350000F2F1E2F0E94453651F110922C0710921C
:102360002D0710922E0710922F071092300710920F
:102370003107109232071092330789A1AC960FB63D
:10238000F894DEBF0FBECDBFDF91CF911F910F91AB
:10239000FF90EF90DF90CF90BF90AF909F908F9085
:1023A0007F906F905F904F903F902F900895809115
:1023B00014078AA3909115079BA3209016073090CD
:1023C0001707409018075090190770901A076090EF
:1023D0001B07CE010D964C01AAA0BBA061017201A2
:1023E000072D162D2CA13EA14FA158A56B2F7A2F9A
:1023F0008F2F9E2F0E94430161E070E082E090E009
:102400000E94490919A2298D3A8D4B8D5C8D6D8DE5
:102410007E8D8F8D98A130584A41564061097109CF
:10242000810991092F37304E424758496240710562
:102430008105910509F008F4A4C082E080933C076F
:1024400020912407309125074091260750912707B6
:10245000609128077091290780912A0790912B0796
:10246000A0E00E944E36F1F184E297E00E9447031B
:102470008AA7A0901407B0901507C0901607D090B7
:102480001707E0901807F090190700911A071091AC
:102490001B07209124073091250740912607509172
:1024A00027076091280770912907CE0101964C01FA
:1024B00080912A0790912B070E9443011F928AA4C2
:1024C000A12CC980DA80EB80FC800D811E812F81D8
:1024D000388549855A856B857C8581E090E00E942E
:1024E000B50D0F90898D80932C078A8D80932D07D1
:1024F0008B8D80932E078C8D80932F078D8D8093ED
:1025000030078E8D809331078F8D8093320788A19D
:1025100080933307A8CE9AA1909314071BA1109320
:10252000150720921607309217074092180750920D
:10253000190770921A0760921B07CE010D964C0185
:10254000A12CB12CC12CD12CE12CF12C00E010E0FD
:102550002CA13EA14FA158A56B2F7A2F8F2F9E2F14
:102560000E9443012AA33BA31A012B01782E692E56
:1025700061E070E082E090E00E94490991E099A357
:1025800042CF88E080933C07ADCFCF93DF93EC013F
:1025900088819981009711F00E94FC361982188277
:1025A0001D821C821B821A82DF91CF910895FC014B
:1025B000808191810C94FC36DC0114964D915C91E4
:1025C00015972091F9063091FA06241B350B261732
:1025D0003707A0F02091F5063091F6062115310558
:1025E00069F0ED91FC91309749F0CB01BF01820F6A
:1025F000931F0E945B3821E0892B09F020E0822F95
:102600000895FC0124813581232B39F421E0FB015D
:102610008081882349F020E007C0808191810E9459
:102620004B3821E0892BB9F7822F0895FC01808176
:102630009181009711F00C94523160E070E0CB0171
:1026400008950F931F93CF93DF938C01EB01FC014F
:10265000808191810097E1F0688179816115710530
:10266000A9F0428153812C813D814217530770F0BC
:102670000E9454388C819D81F801958384831D824A
:102680001C82DF91CF911F910F9108950E94FC361B
:1026900088819981F801918380838A819B819383CA
:1026A00082838C819D8195838483198218821B8209
:1026B0001A82E5CF0F931F93CF93DF93EC018881AC
:1026C0009981009759F02A813B812617370730F00E
:1026D00081E0DF91CF911F910F9108958B016F5F82
:1026E0007F4F0E948537009759F0998388831B8319
:1026F0000A832C813D81232B59F7FC011082E8CFFE
:1027000080E0E7CFEF92FF920F931F93CF93DF9379
:102710006115710541F480E0DF91CF911F910F9118
:10272000FF90EF90089541155105B1F07B01EC0148
:102730000C811D81040F151FB8010E945A138823B4
:1027400051F3288139818C819D81B701820F931FBC
:102750000E9454381D830C8381E0DECFFC01019080
:102760000020E9F73197AF01481B590BBC0181EA02
:1027700096E00C948213EF92FF920F931F93CF93E6
:10278000DF93EC017B018A01BA010E945A13811187
:102790000BC0CE010E94C512CE01DF91CF911F91D7
:1027A0000F91FF90EF9008951D830C83B7018881EE
:1027B00099810E945438F0CFFB0101900020E9F785
:1027C0003197AF01461B570B0C94BB130F931F930C
:1027D000CF93DF93CDB7DEB762970FB6F894DEBF25
:1027E0000FBECDBF8C01FC011182108213821282B8
:1027F000158214824AE0BE016F5F7F4F90E080E057
:102800000E947931BE016F5F7F4FC8010E94DC13C7
:1028100062960FB6F894DEBF0FBECDBFDF91CF91A9
:102820001F910F9108950F931F93CF93DF93CDB70F
:10283000DEB7A2970FB6F894DEBF0FBECDBF8C01F6
:10284000CB01BA01F8011182108213821282158223
:1028500014822AE0AE014F5F5F4F0E948431BE01B7
:102860006F5F7F4FC8010E94DC13A2960FB6F894E9
:10287000DEBF0FBECDBFDF91CF911F910F910895A5
:10288000CF93DF93EC01FB018617970749F0608136
:1028900071816115710541F0448155810E94BB131E
:1028A000CE01DF91CF9108950E94C512F9CFFC01AE
:1028B000118210821382128215821482FB01019010
:1028C0000020E9F73197AF01461B570B0C94BB135F
:1028D000CF92DF92EF92FF920F931F93CF93DF93EC
:1028E0006C017B018A014617570720F48F2D7A016E
:1028F000062F182F6EE174E0C6010E945714C09194
:10290000F906D091FA06EC16FD06F8F40C171D072F
:1029100008F4E801E091F506F091F606EC0FFD1FD2
:10292000108110826091F5067091F6066E0D7F1D84
:10293000C6016115710599F00E94DC138091F506BE
:102940009091F606C80FD91F1883C601DF91CF9169
:102950001F910F91FF90EF90DF90CF9008950E940C
:10296000C512ECCF4F925F926F927F928F929F929F
:10297000AF92BF92CF92DF92EF92FF920F931F938D
:10298000CF93DF93CDB7DEB72C970FB6F894DEBFA9
:102990000FBECDBF62ED71E0CE0107960E945714C5
:1029A00070E060E0CE0107960E94DC1210E0882300
:1029B000A1F061EF71E0CE0101960E94571465E22B
:1029C00070E0CE0101960E94DC1211E0811101C07D
:1029D00010E0CE0101960E94D712CE0107960E9408
:1029E000D712112309F493C381E0809378054DE059
:1029F00050E062E070E0CE0101960E946814BE01D2
:102A00006F5F7F4F8FEE96E00E942113CE010196FB
:102A10000E94D7128FEE96E00E9416136093600119
:102A200070936101809362019093630160317742FA
:102A300081059105E4F480917305811118C080E14E
:102A400097E2A0E0B0E08093600190936101A093D1
:102A50006201B093630165ED71E08CEE95E00E9438
:102A6000D90B64E670E080E090E00E94C20680919D
:102A7000600190916101A0916201B0916301813880
:102A8000934CA94CB140E4F080917305811118C0BA
:102A900080E893ECA9ECB1E0809360019093610130
:102AA000A0936201B093630164EE71E08CEE95E057
:102AB0000E94D90B64E670E080E090E00E94C206BC
:102AC0008091600190916101A0916201B0916301D8
:102AD00080936F0590937005A0937105B093720574
:102AE0004EE150E06DE170E0CE0101960E94681465
:102AF000BE016F5F7F4F87ED96E00E942113CE01EC
:102B000001960E94D71287ED96E00E9416136093FB
:102B10006505613009F0DDC06BED72E087ED96E090
:102B20000E94DC1341E250E060E270E0CE010196C9
:102B30000E946814BE016F5F7F4F89EB96E00E9490
:102B40002113CE0101960E94D71289EB96E00E94D4
:102B50001613162F60936E0548E150E067E170E0B0
:102B6000CE0101960E946814BE016F5F7F4F83EE15
:102B700096E00E942113CE0101960E94D71283EEA7
:102B800096E00E9416136093E90449E150E068E181
:102B900070E0CE0101960E946814BE016F5F7F4F06
:102BA0008DED96E00E942113CE0101960E94D7126E
:102BB0008DED96E00E9416136093E80441E150E029
:102BC0006DE070E0CE0101960E946814BE016F5F57
:102BD0007F4F85E996E00E942113CE0101960E9465
:102BE000D71242E150E061E170E0CE0101960E940F
:102BF0006814BE016F5F7F4F8FEB96E00E94211338
:102C0000CE0101960E94D71247E150E062E170E0E8
:102C1000CE0101960E946814BE016F5F7F4F8BEC5E
:102C200096E00E942113CE0101960E94D7128BECF0
:102C300096E00E9416136093E4047093E504809379
:102C4000E6049093E7044DE150E06CE170E0CE01C2
:102C500001960E946814BE016F5F7F4F89EE96E077
:102C60000E942113CE0101960E94D71289EE96E0B0
:102C70000E941613609374058091760590917705F4
:102C8000892B11F01092740580917405813009F040
:102C900044C090914805911108C09091730591111D
:102CA00004C08093480580937505113009F043C036
:102CB0008091EA049091EB04A091EC04B091ED04B2
:102CC0008093600190936101A0936201B0936301CE
:102CD00032C0623019F463EF71E020CF633019F431
:102CE00066EF71E01BCF643019F469EF71E016CF25
:102CF000653019F46CEF71E011CF663019F46FEFA5
:102D000071E00CCF673019F462E072E007CF6930F0
:102D100009F008CF65E072E001CF81110CC080910D
:102D20004805882341F080917305811104C01092F9
:102D300048051092750580917505882309F45AC0DD
:102D40008091E304811120C0809100018823E1F08B
:102D500080914805811106C068E072E08CEE95E034
:102D60000E94D90B2D986091420170914301072E6A
:102D7000000C880B990B0E94C2065C9A2D9A81E088
:102D80008093E304109200010091E1041091E204A9
:102D90000F5F1F4F1093E2040093E10484E10E944F
:102DA0008806BC01990F880B990B0E94FB316B01BF
:102DB0007C0185E10E948806BC01990F880B990B64
:102DC0000E94FB314B015C01AC019B01C701B601C4
:102DD0000E94893487FD6DC061E080E00E948E0909
:102DE0006CE072E081E497E00E94D90B8091750558
:102DF00081111AC08091E3048823B1F08091000111
:102E0000811112C02D986091400170914101072EEF
:102E1000000C880B990B0E94C2065C982D9A81E0E9
:102E2000809300011092E30480917405813009F0D1
:102E3000D4C08091650584508230A0F480916001F7
:102E400090916101A0916201B0916301885F9A4203
:102E5000A109B1098093600190936101A09362017F
:102E6000B09363018091E9048111D5C08091E80499
:102E7000813009F0D0C06EED73E08FEB96E00E94D8
:102E80000113882309F427C38091600190916101A7
:102E9000A0916201B09163014091E4045091E50476
:102EA0006091E6047091E704840F951FA61FB71F79
:102EB0000AC3053011050CF499CF1092E204109268
:102EC000E104A5019401C701B6010E9475332B01ED
:102ED0003C01A7019601C501B4010E9474339B0116
:102EE000AC01C301B2010E94E1336B017C0120E01F
:102EF00030E0A9010E948934181624F0F7FAF09402
:102F0000F7F8F09420E030E040EA50E4C501B40165
:102F10000E945A3220E030EC4FE754E40E94E13343
:102F200029E23CE54FE85DE30E94E1339B01AC01FF
:102F30000E945A3220E030E048E452E40E94E1333B
:102F40004B015C0120E030E040E050E4C701B601F5
:102F50000E9475332B013C01A701960160E070E0EF
:102F600080E89FE30E94E1339B01AC01C301B20101
:102F70000E9475339B01AC0160E070E080E890E452
:102F80000E94E133A50194010E945A324B015C0179
:102F900061E080E00E948E096FE172E081E497E0D9
:102FA0000E94D90B42E0C701B6010E94010B61E00B
:102FB00088E00E948E0964E272E081E497E00E945A
:102FC000D90B61E08BE00E948E0940E0C501B4019D
:102FD0000E94010B68E272E005CF81111CC0809154
:102FE000E90481113CC28091E804811134C28091CE
:102FF000600190916101A0916201B09163018852DA
:103000009342A109B1098093600190936101A0935B
:103010006201B093630180917805882309F45EC052
:103020008091530581115AC081E10E9423060197C6
:1030300009F054C00091760510917705011511052E
:1030400009F04CC080917505811102C00E94DB0B14
:1030500080917505882309F441C08091450581114F
:1030600002C00E94DB0B809145058130B9F560E01C
:1030700080E00E948E096FE272E081E497E00E9496
:10308000D90B90E2E92EF12C8091FF060E94880670
:10309000080F191F21E0E21AF108B1F7B80185E025
:1030A000759567958A95E1F76F5F7140072E000C63
:1030B000880B990B0E94FB312FE135E847E152E480
:1030C0000E94E13342E00E94010B69E372E081E477
:1030D00097E00E94D90B80E20E94C7091092EF048A
:1030E0002C960FB6F894DEBF0FBECDBFDF91CF9107
:1030F0001F910F91FF90EF90DF90CF90BF90AF9016
:103100009F908F907F906F905F904F9008956CE3A9
:1031100072E0CE0107960E94571470E060E0CE0185
:1031200007960E94DC128823A1F061EF71E0CE01C6
:1031300001960E94571468E070E0CE0101960E944B
:10314000DC1211E0811101C010E0CE0101960E9455
:10315000D712CE0107960E94D7121123E1F048E062
:1031600050E065E070E0CE0101960E946814BE0157
:103170006F5F7F4F85EC96E00E942113CE01019690
:103180000E94D71285EC96E00E94161370935F059B
:1031900060935E05A3CF62E472E0CE0107960E94C1
:1031A000571470E060E0CE0107960E94DC1288237D
:1031B000B9F061EF71E0CE0101960E94571465E00D
:1031C00070E0CE0101960E94DC12882329F011E004
:1031D00080917405811110E0CE0101960E94D712F2
:1031E000CE0107960E94D712112309F453C045E07F
:1031F00050E064E070E0CE0101960E946814BE01C8
:103200006F5F7F4F8DEA96E00E942113CE010196F9
:103210000E94D7128DEA96E00E941613662341F0B1
:1032200080916805811104C080915905882369F057
:103230005F9A5E9861E080E00E948E0967E472E028
:1032400081E497E00E94D90B4BCF613041F45F9845
:103250005E9880E00E948E096CE472E0F1CF6230EB
:1032600049F45F9A5E9A61E080E00E948E0961E510
:1032700072E0E6CF633009F031CF5F985E9A61E08B
:1032800080E00E948E0966E572E081E497E00E948A
:10329000D90B24CF6BE572E0CE0107960E9457143C
:1032A00070E060E0CE0107960E94DC128823A1F056
:1032B00061EF71E0CE0101960E9457146DE070E05D
:1032C000CE0101960E94DC1211E0811101C010E0D4
:1032D000CE0101960E94D712CE0107960E94D71206
:1032E000112301F14DE050E063E070E0CE01019662
:1032F0000E946814BE016F5F7F4F87EA96E00E94CC
:103300002113CE0101960E94D71287EA96E00E940F
:1033100016136093EA047093EB048093EC0490938B
:10332000ED04DCCE6EE572E0CE0107960E945714E4
:1033300070E060E0CE0107960E94DC128823A1F0C5
:1033400061EF71E0CE0101960E94571461E070E0D8
:10335000CE0101960E94DC1211E0811101C010E043
:10336000CE0101960E94D712CE0107960E94D71275
:103370001123C9F060E672E08CEE95E00E94D90B53
:1033800060E080E00E948E0966E672E081E497E0EA
:103390000E94D90B6CE271E080E090E00E94C206CE
:1033A0000E94C51A9DCE67E772E0CE0107960E9483
:1033B000571470E060E0CE0107960E94DC1288236B
:1033C000A1F061EF71E0CE0101960E94571461E017
:1033D00070E0CE0101960E94DC1211E0811101C063
:1033E00010E0CE0101960E94D712CE0107960E94EE
:1033F000D7121111D5CF6DE272E0CE0107960E946F
:10340000571470E060E0CE0107960E94DC1288231A
:10341000A1F064EF71E0CE0101960E94571461E0C3
:1034200070E0CE0101960E94DC1211E0811101C012
:1034300010E0CE0101960E94D712CE0107960E949D
:10344000D712112309F44CCE6EE174E085EF96E0BB
:103450000E94DC1345CE813009F0DDCDC8CD81302E
:1034600009F0D9CD8091E804813009F4C0CD8111F3
:10347000D2CDC0906001D0906101E0906201F090E7
:10348000630188E2C81A83E2D80AE108F108C09211
:103490006001D0926101E0926201F09263016EEDF1
:1034A00073E08FEB96E00E9401138823A1F08091D6
:1034B000E4049091E504A091E604B091E7048C0D3A
:1034C0009D1DAE1DBF1D8093600190936101A0936F
:1034D0006201B09363016DE272E08FEB96E00E94AF
:1034E0000113882309F497CD8091600190916101C7
:1034F000A0916201B09163014091E4045091E50410
:103500006091E6047091E704841B950BA60BB70B42
:103510007ACDCF93DF9300D0CDB7DEB78CEE95E0B8
:103520000E94F5041816190634F56EE174E085EF73
:1035300096E00E94DC138CEE95E00E94F5041816CC
:103540001906B4F48CEE95E00E94D30489831A82A4
:1035500041E050E0BE016F5F7F4F85EF96E00E9433
:10356000821361E070E080E090E00E94C206E3CF49
:1035700081E08093EF048091EF0481110E94B214E6
:103580000F900F90DF91CF9108950F931F93CF93DA
:10359000DF9300D0CDB7DEB78CEE95E00E948405B6
:1035A00062ED71E08CEE95E00E94D90B61EF71E065
:1035B0008CEE95E00E94D90B6EE170E080E090E027
:1035C0000E94C2060091790510917A050F5F1F4F86
:1035D00010937A05009379058CEE95E00E94F5042E
:1035E000892BC9F50E311105B1F5809176059091C1
:1035F0007705892B81F58091730581112CC061E0DD
:103600000E948E0969E772E081E497E00E94D90B7D
:1036100080E20E94C7096091450170914601809146
:103620004701909148010E944F0A6EE772E081E4E1
:1036300097E00E94D90B80E20E94C709109278059A
:10364000109274051092750510927A051092790502
:1036500081E08093E0048091790590917A0502974A
:103660004297D8F480917805811117C08091760532
:1036700090917705892B89F48091E004882369F083
:1036800080917305811109C060E00E948E0964E891
:1036900072E081E497E00E94D90B809179059091C6
:1036A0007A054497DCF080917805811117C08091EC
:1036B000760590917705892B89F48091E004882321
:1036C00069F080917305811109C060E00E948E0944
:1036D00065E972E081E497E00E94D90B8CEE95E0F9
:1036E0000E94F5041816190664F51092E0046EE1C4
:1036F00074E085EF96E00E94DC138CEE95E00E946A
:10370000F50418161906B4F48CEE95E00E94D30463
:1037100089831A8241E050E0BE016F5F7F4F85EFE1
:1037200096E00E94821361E070E080E090E00E94E9
:10373000C206E3CF81E08093EF0410927A051092E5
:1037400079058091EF0481110E94B2140F900F90BF
:10375000DF91CF911F910F9108950F931F93CF93F6
:10376000DF938C01EB010E9418338883C801019616
:103770000E9418338983CE01DF91CF911F910F9161
:103780000895CF92DF92EF92FF920F931F93CF9302
:10379000DF93EB017B0124E0E20EF11C8B016C0155
:1037A000C61AD70AC601800F911F0E941833F8016C
:1037B00081938F01EE15FF05A9F7CE01DF91CF911F
:1037C0001F910F91FF90EF90DF90CF900895CF93CE
:1037D000DF93EB010E9418338883CE01DF91CF91F4
:1037E0000895FF920F931F93CF93DF93EC01F62E72
:1037F00008811981C8010E941833F81621F06F2D35
:10380000C8010E942033CE01DF91CF911F910F910B
:10381000FF9008950F931F93CF93DF9300D0CDB700
:10382000DEB78B019A838983FB016081CE0101960B
:103830000E94F11BC8010F900F90DF91CF911F9153
:103840000F910895AF92BF92CF92DF92EF92FF92C5
:103850000F931F93CF93DF9300D0CDB7DEB78B01CB
:103860006B0124E0C20ED11C7B015C01A61AB70AD1
:10387000C5018E0D9F1D9A838983F70161917F0198
:10388000CE0101960E94F11BEC14FD0489F7C801DA
:103890000F900F90DF91CF911F910F91FF90EF90BC
:1038A000DF90CF90BF90AF900895EF92FF920F936B
:1038B0001F93CF93DF9300D0CDB7DEB78C017B0190
:1038C0009A838983FB016081CE0101960E94F11BDE
:1038D0000F5F1F4F1A830983F7016181CE010196A3
:1038E0000E94F11BC7010F900F90DF91CF911F91A4
:1038F0000F91FF90EF900895CF93DF93EC018091AB
:10390000760590917705009709F0DAC180917305EB
:10391000882369F180917805811129C0C130D105D2
:1039200009F0AAC18091600190916101A0916201AA
:10393000B091630140915C0150915D0160915E0125
:1039400070915F01840F951FA61FB71F81152EE090
:10395000920727E2A20727E0B2070CF048C1809344
:10396000600190936101A0936201B0936301809123
:10397000760590917705039751F5C130D10509F08F
:103980002BC28091FB069091FC06A091FD06B091A0
:10399000FE06805C944BA34BBF4F811529EE920726
:1039A00024EAA20725E3B2070CF011C28093FB06BC
:1039B0009093FC06A093FD06B093FE0681E08093F1
:1039C00053056BEF76E08EE190E00E94221C80911F
:1039D0007605909177050497B1F580917405813053
:1039E00091F1C130D10509F01AC28091490190913D
:1039F0004A01A0914B01B0914C0140915C01509162
:103A00005D0160915E0170915F01840F951FA61F9B
:103A1000B71F803823EC920729ECA20721E0B207F8
:103A20000CF0F8C18093490190934A01A0934B0197
:103A3000B0934C0181E08093530569E471E084E127
:103A400090E00E94221C8091760590917705059761
:103A5000B9F4C130D10509F00AC2809139018F5FF4
:103A6000843008F002C28093390181E080935305CD
:103A70000E94F90769E371E088E290E00E940A1C65
:103A800080917605909177050697E1F4C130D105D4
:103A900009F0FAC180914401833008F4F3C18F5FCB
:103AA00080934401809144018A3018F08AE0809329
:103AB000440181E08093530564E471E08CE390E07D
:103AC0000E940A1C8091760590917705079749F529
:103AD000C130D10509F0F6C180915801909159018A
:103AE000A0915A01B0915B018C599F4FAF4FBF4FCE
:103AF000803828E3920721E0A207B1050CF0DDC170
:103B00008093580190935901A0935A01B0935B019F
:103B100081E08093530568E571E086E490E00E94BF
:103B2000221C80917605909177050897D9F4C130D1
:103B3000D10509F0E9C180914201909143010596B8
:103B4000883E23E092070CF0DCC190934301809300
:103B5000420181E08093530562E471E08AE590E0E0
:103B60000E94551C80917605909177050997D9F4AC
:103B7000C130D10509F0E0C180914001909141012F
:103B80000596883E23E092070CF0D3C19093410143
:103B90008093400181E08093530560E471E08FE5FC
:103BA00090E00E94551C80917605909177050A97C8
:103BB00009F0EDC1C130D10509F0D6C1809156019F
:103BC000909157010196843021E092070CF0C9C111
:103BD000909357018093560181E08093530566E5E9
:103BE00071E084E690E0DF91CF910C94551C80E069
:103BF0009EE0A7E2B7E08093600190936101A093FB
:103C00006201B093630180917605909177050297E8
:103C100009F0ADCEC130D10509F0B2C080914D019F
:103C200090914E01A0914F01B091500140915C01E3
:103C300050915D0160915E0170915F01840F951F4D
:103C4000A61FB71F803422E492072FE0A207B10518
:103C50000CF091C080934D0190934E01A0934F01C1
:103C6000B093500181E0809353056DE471E08AE0E8
:103C700090E00E94221C7BCECF3FDC0709F077CE7C
:103C80008091600190916101A0916201B091630106
:103C900040915C0150915D0160915E0170915F0106
:103CA000841B950BA60BB70B813127E29207A10568
:103CB000B1050CF054CE80E197E2A0E0B0E09BCFDC
:103CC000019709F0A0CFC130D10599F5809151013C
:103CD00090915201A0915301B091540140915C0127
:103CE00050915D0160915E0170915F01840F951F9D
:103CF000A61FB71F803823EC920729ECA20721E00A
:103D0000B20794F48093510190935201A093530110
:103D1000B093540181E08093530561E571E082E343
:103D200090E00E94221C6FCF80E893ECA9ECB1E0F8
:103D3000E9CFCF3FDC0771F780915101909152019B
:103D4000A0915301B091540140915C0150915D01EB
:103D500060915E0170915F01841B950BA60BB70B00
:103D6000813127E29207A105B10564F680E197E26F
:103D7000A0E0B0E0C7CF80E492E4AFE0B0E06ACF6B
:103D8000CF3FDC0709F06ECF80914D0190914E013D
:103D9000A0914F01B091500140915C0150915D01A3
:103DA00060915E0170915F01841B950BA60BB70BB0
:103DB000181619061A061B060CF44CCF10924D016A
:103DC00010924E0110924F01109250014BCF80E0A3
:103DD00099EEA4EAB5E3EACDCF3FDC0709F0EECDDA
:103DE0008091FB069091FC06A091FD06B091FE0625
:103DF00080549B44AC44B109813026E4920723EC03
:103E0000A20723E2B2070CF0D1CD80E096E4A3EC48
:103E1000B3E2CCCD80E893ECA9ECB1E003CECF3F88
:103E2000DC0709F007CE8091490190914A01A091E9
:103E30004B01B0914C0140915C0150915D0160914A
:103E40005E0170915F01841B950BA60BB70B81304F
:103E500026E392072EE6A20721E0B2070CF0E2CD9E
:103E600080E096E3AEE6B1E0DDCD83E0FCCDCF3F70
:103E7000DC0709F0FACD80913901815009F0F3CDCA
:103E800081E0F1CD83E00CCECF3FDC0709F011CE0D
:103E900080914401882309F40CCE9EEF980F815045
:103EA000923008F482E08093440180914401833091
:103EB00008F0FFCD10924401FCCD80E898E3A1E02A
:103EC000B0E01ECECF3FDC0709F022CE8091580132
:103ED00090915901A0915A01B0915B0184569109CA
:103EE000A109B109181619061A061B060CF408CE0A
:103EF000109258011092590110925A0110925B01D0
:103F000007CE88EE93E021CECF3FDC0709F021CE2B
:103F10008091420190914301009709F41ACE0597D0
:103F2000181619060CF411CE10924301109242019A
:103F300010CE88EE93E02ACECF3FDC0709F02ACEE0
:103F40008091400190914101009709F423CE05979B
:103F5000181619060CF41ACE109241011092400165
:103F600019CE84E091E034CE219609F035CE8091CF
:103F7000560190915701873C910509F42DCE019788
:103F8000893C91050CF024CE88EC90E021CEDF91A5
:103F9000CF9108951F920F920FB60F9211242F9375
:103FA0003F934F935F936F937F938F939F93AF93C1
:103FB000BF93EF93FF938CEE95E00E941505FF9160
:103FC000EF91BF91AF919F918F917F916F915F9191
:103FD0004F913F912F910F900FBE0F901F9018950A
:103FE0001F920F920FB60F9211242F938F939F93CE
:103FF000EF93FF93E091FC05F091FD058081E09146
:104000000206F091030682FD1BC090818091050697
:104010008F5F8F7320910606821741F0E0910506AD
:10402000F0E0E451FA4F958F80930506FF91EF91F0
:104030009F918F912F910F900FBE0F901F90189509
:104040008081F4CF1F920F920FB60F9211242F93FD
:104050003F938F939F93AF93BF9380913905909136
:104060003A05A0913B05B0913C053091330523E022
:10407000230F2D3758F50196A11DB11D209333054F
:104080008093390590933A05A0933B05B0933C0586
:104090008091340590913505A0913605B091370592
:1040A0000196A11DB11D8093340590933505A09311
:1040B0003605B0933705BF91AF919F918F913F9196
:1040C0002F910F900FBE0F901F90189526E8230F89
:1040D0000296A11DB11DD2CF1F920F920FB60F9263
:1040E00011242F933F934F935F936F937F938F93FD
:1040F0009F93AF93BF93EF93FF938091B900887F15
:10410000803609F44AC0F0F5883209F4A7C018F5E2
:10411000803109F49BC0B8F4882309F4F9C08830D1
:1041200009F494C0FF91EF91BF91AF919F918F914E
:104130007F916F915F914F913F912F910F900FBEA3
:104140000F901F901895883109F488C0803251F77C
:104150008093C50514C0803409F49DC040F48033B9
:10416000B9F38833F9F68093C50585ECB0C0803586
:1041700009F485C0883509F496C0883499F60E9400
:10418000F506D0CF883909F48CC038F5883729F086
:1041900050F4883611F0803729F683E08093C70504
:1041A0001092320557C0883809F47BC0803919F065
:1041B000803809F0B7CF80913205803208F071C0A5
:1041C000E091320581E08E0F809332058091BB0033
:1041D000F0E0EE5EFA4F80833DC0803B39F0E0F4C2
:1041E000803A09F479C0883A09F09CCF84E0809342
:1041F000C7051092110510921005E0917D05F09110
:104200007E0509958091100581110FC081E0809392
:1042100010051092F00409C0803C09F4A6CF883C38
:1042200009F4A3CF883B09F07DCFE091110581E02F
:104230008E0F80931105F0E0E051FB4F8081809359
:10424000BB00909111058091100529C08091A205B5
:104250008093BB0085EC8093BC0064CF9091C40533
:104260008091C305981758F5E091C40581E08E0F41
:104270008093C405F0E0ED55FA4F8081E9CFE091DD
:10428000C40581E08E0F8093C4058091BB00F0E0EF
:10429000ED55FA4F80839091C4058091C30598171E
:1042A000C8F285E8D8CFE091C40581E08E0F8093F5
:1042B000C4058091BB00F0E0ED55FA4F80838091FA
:1042C000C60581115CCF81E08093A10584EA8093CB
:1042D000BC001092C70526CF85EC8093BC001092DD
:1042E000C70580913205803230F4E0913205F0E06C
:1042F000EE5EFA4F10826091320570E0E0917B052E
:10430000F0917C0582E195E00995109232050ACF83
:104310001092C50534CF1F920F920FB60F92112441
:104320002F933F934F935F936F937F938F939F93BD
:10433000AF93BF93CF93DF93EF93FF9380910207E7
:104340000E942306EC01809101070E9423069091B0
:1043500000079F70CC0FDD1FC82B24E0929FC00187
:10436000112486589E4FC80FD92FD11D8881809364
:104370000007807371F08031F9F481E090E00E94D1
:104380007C1C809176059091770568ED74E0892B0F
:1043900009F1FF91EF91DF91CF91BF91AF919F9183
:1043A0008F917F916F915F914F913F912F910F90DE
:1043B0000FBE0F901F901895803259F78FEF9FEF27
:1043C0000E947C1C8091760590917705892B09F7D6
:1043D0006CED74E08CEE95E00E94D90BDACFAF92D1
:1043E000BF92CF92DF92EF92FF920F931F93CF93E2
:1043F000DF93ECEEF5E01382128288EE93E0A0E00A
:10440000B0E084839583A683B7832AE931E03183C2
:10441000208325EC30E03587248724EC30E0378793
:10442000268720EC30E0318B208B21EC30E0338B81
:10443000228B22EC30E0358B248B26EC30E0378B5E
:10444000268B118E128E138E148EE9E8F6E01382FD
:10445000128284839583A683B7838CEA91E091834B
:104460008083E1E4F7E0138212828EEB91E0918386
:10447000808387E2848380E1818782E0828713865C
:10448000E3E0F7E098E090AF91AF11AA12AA13AA67
:104490001186128613861486158616861786108A4C
:1044A000118A128A138A148A158A168A178A108E1C
:1044B000118E128E138E148E158E168E178E10A2DC
:1044C00011A212A213A214A215A216A217A210A63C
:1044D00011A612A613A614A615A616A617A610AA0C
:1044E00040ED50E967EF71E042AF53AF64AF75AF95
:1044F000C0E0D7E0898383E08A8360E082E00E94A5
:104500004C0660E08A810E944C0689810E94CD059C
:104510008A810E94CD0518828FE08093FF0620914A
:10452000640130916501409166015091670160918D
:1045300068017091690180916A0190916B01E4E6D4
:10454000AE2EB12CC12CD12CE12CF12C00E010E0CE
:104550000E9499352093FB063093FC064093FD069C
:104560005093FE066EE174E085EF96E00E945714CA
:104570006EE174E08FEE96E00E9457146EE174E0F5
:1045800089EE96E00E9457146EE174E083EE96E0A7
:104590000E9457146EE174E08DED96E00E9457146E
:1045A00066EA72E087ED96E00E9457146EE174E0CF
:1045B00081ED96E00E9457146EE174E08BEC96E07A
:1045C0000E9457146EE174E085EC96E00E94571447
:1045D0006EE174E08FEB96E00E9457146EE174E098
:1045E00089EB96E00E9457146EE174E083EB96E04D
:1045F0000E9457146EE174E08DEA96E00E94571411
:104600006EE174E087EA96E00E9457146EE174E070
:1046100081EA96E00E9457146EE174E08BE996E01F
:104620000E9457146EE174E085E996E0DF91CF9126
:104630001F910F91FF90EF90DF90CF90BF90AF90C0
:104640000C945714CF93DF93CDB7DEB72C970FB6EA
:10465000F894DEBF0FBECDBF789484B5826084BD70
:1046600084B5816084BD85B5826085BD85B5816076
:1046700085BD80916E00816080936E0010928100F4
:1046800080918100826080938100809181008160AF
:104690008093810080918000816080938000809170
:1046A000B10084608093B1008091B00081608093FC
:1046B000B00080917A00846080937A0080917A00C3
:1046C000826080937A0080917A00816080937A0082
:1046D00080917A00806880937A001092C10060E037
:1046E0008FE00E944C0661E084E00E944C0660E08E
:1046F00085E00E944C0661E086E00E944C0661E085
:1047000087E00E944C0661E088E00E944C0661E070
:1047100089E00E944C0661E08AE00E944C0661E05C
:104720008BE00E944C0661E08CE00E944C0661E048
:104730008DE00E944C0660E08EE00E944C0660E036
:104740008FE00E944C0660E080E10E944C0660E031
:1047500081E10E944C0660E08EE00E944C0660E021
:104760008FE00E944C0660E080E10E944C0660E011
:1047700081E10E944C0660E084E10E944C0660E00A
:1047800085E10E944C0662E085E00E944C060E9492
:10479000F3051092460780914B07823018F098E09D
:1047A000909346078093490762E370E080E090E0D1
:1047B0000E94C20660914C0781E497E00E94E307E3
:1047C00068EE73E080E090E00E94C20660E381E45E
:1047D00097E00E945E090BE416E4C8010197F1F727
:1047E00060E381E497E00E945E09C8010197F1F758
:1047F00060E381E497E00E945E0983E592E001971F
:10480000F1F760E281E497E00E945E09609146075B
:10481000606240E081E497E00E94770984E0809341
:10482000470740E06CE081E497E00E9477090E942E
:10483000D00982E08093480740E066E081E497E099
:104840000E94770940E062E081E497E00E947709E6
:104850008BE39FE10197F1F788E080934C0760E0DC
:1048600081E497E00E94E30768E375E090E080E070
:104870000E94E71BFC018081883C09F40BC388EC93
:1048800090E09A838983BE016F5F7F4F90E080E064
:104890000E94551C6DE471E08AE090E00E94221CA9
:1048A00069E471E084E190E00E94221C6BEF76E005
:1048B0008EE190E00E94221C69E371E088E290E0C2
:1048C0000E940A1C61E571E082E390E00E94221CD4
:1048D00064E471E08CE390E00E940A1C68E571E0FA
:1048E00086E490E00E94221C65E475E080E590E09B
:1048F0000E940A1C62E471E08AE590E00E94551C67
:1049000060E471E08FE590E00E94551C66E571E07F
:1049100084E690E00E94551C6DE471E08AE090E02E
:104920000E94C11BFC0180819181A281B38180938F
:104930004D0190934E01A0934F01B093500169E453
:1049400071E084E190E00E94C11BFC0180819181B3
:10495000A281B3818093490190934A01A0934B01B6
:10496000B0934C016BEF76E08EE190E00E94C11BAA
:10497000FC0180819181A281B3818093FB06909399
:10498000FC06A093FD06B093FE0669E371E088E2A1
:1049900090E00E94E71BFC0180818093390161E572
:1049A00071E082E390E00E94C11BFC018081918153
:1049B000A281B3818093510190935201A09353013E
:1049C000B093540164E471E08CE390E00E94E71B33
:1049D000FC0180818093440168E571E086E490E009
:1049E0000E94C11BFC0180819181A281B3818093CF
:1049F000580190935901A0935A01B0935B0165E46B
:104A000075E080E590E00E94E71BFC0180818093C7
:104A1000450562E471E08AE590E00E94AD1BFC016F
:104A200080819181909343018093420160E471E021
:104A30008FE590E00E94AD1BFC01808191819093F5
:104A400041018093400166E571E084E690E00E94B8
:104A5000AD1BFC0180819181909357018093560199
:104A60000E94F9070E94A5088091680084608093E5
:104A7000680080916D008C6080936D00789461E394
:104A800071E081E00E94DB0969E271E082E00E944E
:104A9000DB0961E271E083E00E94DB0969E171E01A
:104AA00084E00E94DB0961E171E085E00E94DB099E
:104AB00069E071E086E00E94DB0961E071E087E077
:104AC0000E94DB096091FB067091FC068091FD0657
:104AD0009091FE0624E630E040E050E00E942C3544
:104AE0002093640130936501409366015093670100
:104AF000609368017093690180936A0190936B01E0
:104B000080914D0190914E01A0914F01B0915001C3
:104B10008093370790933807A0933907B0933A07EB
:104B2000C0904901D0904A01E0904B01F0904C01B7
:104B30000E94F30562E987EB0E94A507C114D10426
:104B4000E104F104D1F08FE00E94CB08682F6F736D
:104B5000F1E8CF16F3ECDF06F9ECEF06F1E0FF0623
:104B600008F09FC1C0923D07D0923E07E0923F07F8
:104B7000F09240078FE00E94A50760E880E10E9464
:104B8000A50760E881E10E94A50760E882E10E9434
:104B9000A5076CE080E10E94A5076CE081E10E941E
:104BA000A5076CE082E10E94A50760E281EB0E940C
:104BB000A50760E881EB0E94A50720916401309170
:104BC00065014091660150916701609168017091A3
:104BD000690180916A0190916B0110E000E00E94F0
:104BE000050C80E10E94CB08682F636080E10E9481
:104BF000A5072D9A60E080E00E948E0969EA72E0C4
:104C000081E497E00E94D90B61E080E00E948E0968
:104C10006AEB72E081E497E00E94D90B68EE73E0E2
:104C200080E090E00E94C20618E0212E312C0E9404
:104C3000C51A8091790590917A054F9720F01092CE
:104C40007A0510927905809178058823D9F08091B2
:104C5000760590917705892BA9F4809161058111E2
:104C600011C08091730581110DC08091750581116E
:104C70004EC160E00E948E096BEC72E081E497E027
:104C80000E94D90B8EE00E94880690934305809382
:104C900042058438934044F080916405811104C03A
:104CA00010926305109241058EE00E948806909351
:104CB0004305809342052FB7F89480913905909170
:104CC0003A05A0913B05B0913C052FBF0197A10982
:104CD000B10985369105A105B10510F18EE00E945C
:104CE00088062091420530914305AC01435051099B
:104CF0002417350744F003968217930724F0309366
:104D0000400520933F0500913F051091400505386F
:104D100023E012070CF405C11092440510926405BB
:104D200080E10E942306892BF9F480914A058111C4
:104D30001BC080917305811117C0809149058111B5
:104D400013C08091670581110FC0809148058111C2
:104D50000BC081E080934A058093750568E072E09E
:104D60008CEE95E00E94D90B80E10E94230601970A
:104D700071F480914A05882351F010924A051092EF
:104D8000750565ED72E08CEE95E00E94D90B81E12E
:104D90000E942306892B09F02DC2809147058111BD
:104DA00029C280917505811125C2809173058111F9
:104DB00021C2009176051091770581E08093470527
:104DC0000F5F1F4F10937705009376050E94D0095F
:104DD0000130110509F00BC28091600190916101D1
:104DE000A0916201B0916301885D9C4DAF4FBF4FB0
:104DF00080933C0190933D01A0933E01B0933F010D
:104E000067ED76E081ED96E00E94401480914405C4
:104E10008111F0C167ED76E081ED96E00E944014CB
:104E200061E571E082E390E00E94C11BFC014081DA
:104E3000518162817381409351015093520160937B
:104E4000530170935401CE0107960E9413148B8571
:104E50009C850B9708F0BFC4CE0101960E94E61313
:104E60004B855C856F817885CE0101960E94821307
:104E7000811104C0CE0101960E94C512BE016F5F70
:104E80007F4FCE0107960E944014CE0101960E94EA
:104E9000D712DDCF81E10E942306892B09F4EFCCE4
:104EA0003BCDD701C6018158934CA94CB140803805
:104EB000934CA94CB14070F4F694E794D794C794FE
:104EC000C0923D07D0923E07E0923F07F092400724
:104ED000606450CED701C60181509748A349B340C2
:104EE00081159A45A246B24008F044CE02E0F694FD
:104EF000E794D794C7940A95D1F7C0923D07D09212
:104F00003E07E0923F07F0924007606833CE809101
:104F100045058111B7CE60E00E948E0960ED72E018
:104F2000ADCE0F311105A4F580913E059091640539
:104F300091112EC081111EC080915305811128C08E
:104F400080917305811124C080917805882301F137
:104F50008091480581111CC011E010933E0510930B
:104F6000640568E072E08CEE95E00E94D90B109326
:104F70007505D6CE10923E0581E0809364051092AF
:104F8000750565ED72E08CEE95E00E94D90BC8CEF8
:104F9000C8018F978A9748F580916405811125C0D3
:104FA00080913E05811121C080914A0581111DC06B
:104FB00080913A01815080933A01809176059091D9
:104FC0007705892B71F469ED72E085E996E00E941E
:104FD0000113811106C060E672E08CEE95E00E943C
:104FE000D90B81E0809364059BCEC8018A55910955
:104FF000C49710F58091640581111EC080913E0513
:1050000081111AC080914A05811116C080913A0120
:105010008F5F80933A018091760590917705892B77
:1050200001F76EED72E085E996E00E94011363EEF0
:1050300072E08111D6CFD1CFC8018F5891098D97D9
:1050400020F580916405811120C080913E05811179
:105050001CC080914A05811118C0809153058111AF
:1050600014C0809176059091770569EE72E0892BE6
:1050700009F0B7CF8CEE95E00E94D90B62E370E0A7
:1050800080E090E00E94C206ACCFC8018D5B910920
:105090008B97C8F480916405811115C080913E05FD
:1050A000811111C080914A0581110DC08091530575
:1050B000811109C06DEE72E083EB96E00E9401134E
:1050C000882309F455C0C801895E91098A9708F4BC
:1050D00059C0045111400C32110508F021CE8091C5
:1050E000640581111DCE80917505811119CE8091C5
:1050F0004105811115CE81E08093640580934105BF
:1051000080913D058F5F80933D05813031F460E0F3
:1051100073E08CEE95E00E94D90B80913D058230C2
:1051200031F467E073E08CEE95E00E94D90B80913A
:105130003D05833031F46EE073E08CEE95E00E9423
:10514000D90B80913D05843031F465E173E08CEE3C
:1051500095E00E94D90B80913D05843010F01092AB
:105160003D056AE070E080E090E00E94C206D8CD84
:105170008091760590917705892B09F032CF61EF08
:1051800072E078CF809175058111A3CF809163057E
:1051900081119FCF80917805882309F49ACF11E07F
:1051A0001093640510936105809162058F5F809371
:1051B0006205843108F4B4CD60E080E00E948E097D
:1051C00065EF72E081E497E00E94D90B6AEF72E02C
:1051D0008CEE95E00E94D90B6AE070E080E090E0F0
:1051E0000E94C206109262051093630599CD012BAF
:1051F00009F00CCE81E10E942306019751F48091C1
:105200004705882331F080917305811102C0109207
:10521000470500917605109177050130110539F4A5
:1052200080916705811103C081E08093670585E067
:105230000E942306019761F480914605811108C000
:1052400080913B0191E0892780933B019093460533
:1052500085E00E942306892BB1F4809146058823BE
:1052600091F08091750581110EC00115110559F459
:105270001092460580913B018111FCC681E080932C
:1052800073058093490585E00E942306892BC9F4A4
:10529000809146058823A9F080917505882389F0BF
:1052A000012B79F41092460580913B018111EFC6E4
:1052B00081E08093450565E475E080E590E00E941B
:1052C0000A1C00917605109177050115110509F466
:1052D00040C38091750581113CC30E943C08013098
:1052E000110509F052C061E571E082E390E00E948F
:1052F000C11BFC01608171818281938160935101A6
:1053000070935201809353019093540160934F0521
:1053100070935005809351059093520520E432E438
:105320004FE050E00E94B53420934B0530934C057C
:1053300040934D0550934E0560E080E00E948E0939
:1053400067E273E081E497E00E94D90B0E94790A3A
:1053500061E080E00E948E0968EF73E081E497E0ED
:105360000E94D90B60915C0170915D0180915E019A
:1053700090915F010E944F0A6DE273E081E497E033
:105380000E94D90B80E20E94C70980917605909116
:105390007705029709F071C061E571E082E390E062
:1053A0000E94C11BFC0180819181A281B381809305
:1053B000510190935201A0935301B093540160E0C6
:1053C00080E00E948E0962E373E081E497E00E942E
:1053D000D90BC0905101D0905201E0905301F09050
:1053E0005401F8E2CF1AF3E2DF0AE108F108B2E073
:1053F000CC0CDD1CEE1CFF1CBA95D1F7C701B60121
:1054000020E432E44FE050E00E94B53420934B0595
:1054100030934C0540934D0550934E05C0924F0577
:10542000D0925005E0925105F09252050E94790AFF
:1054300061E080E00E948E0968E373E081E497E018
:105440000E94D90B60915C0170915D0180915E01B9
:1054500090915F010E944F0A61E08AE00E948E09EC
:1054600060914D0170914E0180914F0190915001DA
:105470000E944F0A80E20E94C709809176059091B0
:105480007705039731F560E082E00E948E096EE3B4
:1054900073E081E497E00E94D90B61E086E00E940E
:1054A0008E096091FB067091FC068091FD0690913B
:1054B000FE0620E432E44FE050E00E94B534CA0119
:1054C000B9010E944F0A6DE473E081E497E00E9405
:1054D000D90B80917605909177050497F1F460E0FF
:1054E00080E00E948E0962E573E081E497E00E940B
:1054F000D90B61E084E00E948E09609149017091AE
:105500004A0180914B0190914C010E944F0A63E641
:1055100073E081E497E00E94D90B80917605909129
:105520007705059709F560E080E00E948E0967E63F
:1055300073E081E497E00E94D90B61E083E00E9470
:105540008E0967E773E081E497E00E94D90B6091D0
:1055500045017091460180914701909148010E9458
:105560004F0A80E20E94C7098091760590917705E5
:10557000069759F564E471E08CE390E00E94E71B24
:10558000FC0180818093440160E081E00E948E09EB
:105590006EE773E081E497E00E94D90B80914401AB
:1055A00061E0882309F448C187E00E948E09609178
:1055B000440170E090E080E04AE00E94090A6EE851
:1055C00073E081E497E00E94D90B80917605909179
:1055D0007705079709F560E080E00E948E096AE987
:1055E00073E081E497E00E94D90B61E085E00E94BE
:1055F0008E09609158017091590180915A019091E2
:105600005B010E944F0A6DE273E081E497E00E9423
:10561000D90B80E20E94C7098091760590917705A9
:10562000089711F560E082E00E948E096BEA73E052
:1056300081E497E00E94D90B80914201909143014F
:1056400060E0892B09F406C18AE00E948E0960910E
:10565000420170914301072E000C880B990B0E94A8
:105660004F0A80E20E94C7098091760590917705E4
:10567000099711F560E082E00E948E0960EC73E00A
:1056800081E497E00E94D90B809140019091410103
:1056900060E0892B09F4F2C08AE00E948E096091D3
:1056A000400170914101072E000C880B990B0E945C
:1056B0004F0A80E20E94C709809176059091770594
:1056C0000A9709F052C08091560190915701843099
:1056D000914074F560E081E00E948E0965ED73E011
:1056E00081E497E00E94D90B60E08BE00E948E0974
:1056F00060915601709157016A587109072E000C8C
:10570000880B990B0E94FB3120E030E040E05FE322
:105710000E945A320E945334072E000C880B990BBA
:105720000E944F0A60EE73E081E497E00E94D90B7B
:10573000809156019091570184309140B4F060E01F
:1057400081E00E948E0964EE73E081E497E00E949C
:10575000D90B80E20E94C70980E20E94C70984E059
:1057600091E0909357018093560180917605909136
:1057700077050B970CF4EDC040913C0150913D0131
:1057800060913E0170913F01CE0107960E94131473
:105790008B859C850B9708F085C0CE0101960E94F1
:1057A000E6134B855C856F817885CE0101960E945A
:1057B0008213811104C0CE0101960E94C512BE0160
:1057C0006F5F7F4FCE0107960E944014CE01019675
:1057D0000E94D712DDCF6CE173E08CEE95E00E9461
:1057E000D90BBE01695F7F4F8CEE95E00E94890462
:1057F00061EF71E08CEE95E00E94D90B6FE173E0F0
:105800008CEE95E00E94D90B80915101909152014C
:10581000A0915301B0915401809360019093610174
:10582000A0936201B093630181E080934405CE01AF
:1058300007960E94D712DECC87E00E948E0964E9A9
:1058400073E081E497E00E94D90B109266051092F4
:105850004401BBCE82E00E948E0964EB73E081E4D8
:1058600097E00E94D90B80E20E94C70980E20E9463
:10587000C7091092430110924201F6CE82E00E94C5
:105880008E0969EC73E081E497E00E94D90B80E215
:105890000E94C70980E20E94C7091092410110923C
:1058A00040010ACF6CE173E08CEE95E00E94D90BC9
:1058B000BE01695F7F4F8CEE95E00E94890461EF25
:1058C00071E08CEE95E00E94D90B62EF73E08CEEF4
:1058D00095E00E94D90B61ED76E08CEE95E00E9498
:1058E000890461EF71E08CEE95E00E94D90B6EE1C6
:1058F00074E081ED96E00E94DC138CEE95E00E944E
:10590000840562E471E08AE590E00E94AD1BFC0131
:1059100080819181909343018093420160E471E022
:105920008FE590E00E94AD1BFC01808191819093F6
:105930004101809340011092530510926705109227
:105940007705109276050E94D009CE0107960E9435
:10595000D71280917805811139C010927405109288
:10596000750580917305882389F10E943C08809118
:10597000600190916101A0916201B09163018093F7
:105980006F0590937005A0937105B09372050E9406
:10599000DB0B61E080E00E948E0967EF73E081E439
:1059A00097E00E94D90B60915C0170915D0180913C
:1059B0005E0190915F010E944F0A6EEF73E081E4F7
:1059C00097E00E94D90B80E20E94C709809176057A
:1059D00090917705892B09F0DEC1809175058111C1
:1059E0007FC080917305882309F45BC040906001FB
:1059F0005090610160906201709063018091540544
:105A000090915505A0915605B09157054816590635
:105A10006A067B0609F445C01091780561E082E0D2
:105A200090E00E943109A0906401B0906501C0909F
:105A30006601D0906701E0906801F09069010091E3
:105A40006A01112309F426C310916B01C301B2014D
:105A5000685D7C4D8F4F9F4F24E630E040E050E082
:105A60000E942C35A2E08A2E912C0E94710E60E0DB
:105A700080E00E948E0966E074E081E497E00E9475
:105A8000D90B8091600190916101A0916201B09168
:105A900063018093540590935505A0935605B093E8
:105AA000570510917305111105C060E082E090E088
:105AB0000E94310980917805882309F4F0C21123EE
:105AC00059F080915305811107C01092690561E07A
:105AD00090E080E00E943109809175058823B1F043
:105AE00080916E05813091F48CEE95E00E948405E2
:105AF0006AE074E08CEE95E00E94D90B65E070E0FE
:105B000080E090E00E94C2060E94891A8091780588
:105B1000882309F440C18091750581113CC18091B1
:105B200058058F5F853009F47DC0809358056EE17C
:105B300074E081EA96E00E94DC1300915E0510910A
:105B40005F05013811050CF47EC089E090E0909368
:105B50005D0580935C050A3811050CF0BCC080918E
:105B60005601909157018430E1E09E0714F5081723
:105B700019073CF020915905211103C021E0209321
:105B8000590520915905222359F0209155012223CE
:105B900039F08897081719071CF4215020935501F4
:105BA00080915501811105C08FE0809355011092BD
:105BB000590580915C0590915D05893091050CF443
:105BC000A0C085E194E00E94AE1361E08DE00E94E8
:105BD0008E0980915A0590915B05181619069CF460
:105BE0006EED73E081E497E00E94D90B60915A0555
:105BF00070915B05072E000C880B990B0E944F0AD1
:105C000080E20E94C70980915A0590915B051816A1
:105C100019060CF47EC06BE274E081E497E00E9408
:105C2000D90B77C0109258056EE074E08CEE95E0C9
:105C30000E94D90B65E070E080E090E00E94C2060F
:105C40000E94891A74CF043111052CF410925D055D
:105C500010925C0584CFC80144974B9738F481E0DB
:105C600090E090935D0580935C0579CFC8018F9794
:105C7000E2E0F0E00D97E8F0C801CC970B9718F43C
:105C800083E090E0EECFC80187549109E4E0F0E0B2
:105C90000A9778F0C801815591090C9718F485E0AE
:105CA00090E0DFCFC8018D5591090B9738F4E6E0FD
:105CB000F0E0F0935D05E0935C0551CFC801885694
:105CC00091090B9718F487E090E0CBCF30925D05F7
:105CD00020925C0544CFB8016A587109072E000C68
:105CE000880B990B0E94FB3120E030E040E05FE33D
:105CF0000E945A320E94533470935B0560935A0598
:105D00002ECF8830910509F0E0C08FE194E00E9429
:105D1000AE1361E084E00E948E0961EA76E081E4DE
:105D200097E00E948904809160058F5F863009F4B6
:105D3000F8C0809360058091640581112CC080912A
:105D40006305811128C080916205883220F5809119
:105D50006105882301F160E080E00E948E0965EB17
:105D600074E081E497E00E94D90B6CE271E080E07E
:105D700090E00E94C2066AEB74E08CEE95E00E940F
:105D8000D90B6AE070E080E090E00E94C2061092B9
:105D90006105109262058091600190916101A0916E
:105DA0006201B091630140916A0550916B05609169
:105DB0006C0570916D0584179507A607B70721F04C
:105DC00020916905222339F02091760530917705DD
:105DD000232B09F458C0AC01BD0140515742610961
:105DE00071094035514F6242710508F0ABC02C9AE1
:105DF0002B982A98299828986DEE72E083EB96E00C
:105E00000E94DC134090600150906101609062013B
:105E1000709063018091780581114DC18091760564
:105E200090917705892B39F1A0906401B0906501BC
:105E3000C0906601D0906701E0906801F090690120
:105E400000916A0110916B01C301B2016852734263
:105E500081099109F2E0660F771F881F991FFA9553
:105E6000D1F724E630E040E050E00E942C35912C40
:105E7000812C0E94710E40926A0550926B056092CF
:105E80006C0570926D052091B7063091B80680912F
:105E90009F069091A0062817390709F02CC1809120
:105EA000B3069091B40660919B0670919C06009792
:105EB00009F414C16115710509F0D9C0232B09F447
:105EC00042C1FC01808190E014C18730910519F432
:105ED0008FE294E01CCF8630910519F48FE394E0B3
:105EE00016CF8530910519F48FE494E010CF8430FB
:105EF000910519F48FE594E00ACF8330910519F4E8
:105F00008FE694E004CF8230910519F48FE794E096
:105F1000FECE019719F48FE894E0F9CE8FE994E072
:105F2000F6CE109260056FEA74E08CEE95E00E9468
:105F3000D90B65E070E080E090E00E94C2060E940C
:105F4000891AF9CEAC01BD0140565841634271092E
:105F5000403854486E41710540F42C982B9A2A9889
:105F60002998289860EC74E049CFAC01BD01405EEF
:105F70005C4961447109403255476843710540F4FA
:105F80002C982B982A9A2998289863EC74E036CF9D
:105F9000AC01BD0152516A477109411559406D4329
:105FA000710540F42C982B982A98299A289866EC29
:105FB00074E024CFAC01BD015B51674B7109411501
:105FC00059406D43710540F42C982B982A98299AD2
:105FD000289869EC74E012CFAC01BD015452644FB3
:105FE0007109403C564C6D42710540F42C982B9839
:105FF0002A982998289A6CEC74E000CFAC01BD0176
:10600000405C5A4E61427140403C564C6D427105B5
:1060100040F42C982B982A982998289A6FEC74E0D1
:10602000EDCEAC01BD014058514B6F44714040343E
:106030005B446C44710548F42C982B982A98299855
:10604000289A289A62ED74E0D9CE805C9C4FAB49C7
:10605000B140813C964CAD42B10508F0D3CE2C98AE
:106060002B982A982998289A65ED74E0C7CE0E944B
:106070004B383FC010927305109249051092540599
:10608000109255051092560510925705FCC81092B3
:10609000450511C910916B01C301B201DDCC80919E
:1060A0005305112309F40FCD811116CD81E08093A2
:1060B000690560E00DCDA0906401B0906501C090CD
:1060C0006601D0906701E0906801F090690100914D
:1060D0006A0110916B01C301B201BCCE611571055B
:1060E00091F1232B81F1FB01808190E091958195C5
:1060F0009109892B41F180916E05811124C0809115
:106100006805811120C08091750581111CC08091A6
:106110007305811118C080916705811114C066E66E
:1061200075E08CE390E00E94E71BFC018081809386
:1061300066050E94A50861E081E090E00E943109B7
:1061400081E080936805809166058823D1F1909164
:1061500068059923B1F1815080936605A090640190
:10616000B0906501C0906601D0906701E090680131
:10617000F090690100916A0110916B0160916001DA
:10618000709161018091620190916301409058018A
:106190005090590160905A0170905B01640D751D1B
:1061A000861D971D685D7C4D8F4F9F4F24E630E024
:1061B00040E050E00E942C3588248394912C0E946A
:1061C000710E80916605882361F0809168058823AF
:1061D00041F080917505811104C080917305882379
:1061E00039F060E081E090E00E943109109268058A
:1061F00063EB76E08BE996E00E94401480E090E04B
:10620000892B11F40C9417260E940105882311F4A0
:106210000C9417260E9400000C94172685E996E03E
:106220000E94D7128BE996E00E94D71281EA96E08D
:106230000E94D71287EA96E00E94D7128DEA96E074
:106240000E94D71283EB96E00E94D71289EB96E06A
:106250000E94D7128FEB96E00E94D71285EC96E051
:106260000E94D7128BEC96E00E94D71281ED96E047
:106270000E94D71287ED96E00E94D7128DED96E02E
:106280000E94D71283EE96E00E94D71289EE96E024
:106290000E94D7128FEE96E00E94D71285EF96E00B
:1062A0000C94D7121F93FC0199278827BC01E8940E
:1062B00011911032E9F3193010F01E30C8F31B327F
:1062C00051F01D3249F4689406C00E949331610F69
:1062D000711D811D911D119110531A30B0F33EF4C0
:1062E00090958095709561957F4F8F4F9F4F1F912F
:1062F0000895BB274A3031F4992322F4BDE29095EA
:1063000081959F4F0C94CB31BB272A3051F49923B0
:1063100042F4BDE290958095709561957F4F8F4FC7
:106320009F4F0C94A931592F482F372F262F660FD6
:10633000771F881F991F660F771F881F991F620F8D
:10634000731F841F951F660F771F881F991F08955D
:10635000BB27FA01A62F6217710581059105330B42
:1063600030FB66F0AA27660F771F881F991FAA1FA8
:10637000A21710F0A21B63953850A9F7A05DAA33AD
:1063800008F0A95DA19336F7B111B1931082CA014B
:106390000C94E431BB27FB015527AA27880F991FCE
:1063A000AA1FA41710F0A41B83955051B9F7A05D44
:1063B000AA3308F0A95DA193009779F7B111B193C1
:1063C0001192CB010C94E431DC01FC01672F719137
:1063D0007723E1F7329704C07C916D9370836291CB
:1063E000AE17BF07C8F308950E94363208F481E063
:1063F0000895E89409C097FB3EF4909580957095B8
:1064000061957F4F8F4F9F4F9923A9F0F92F96E900
:10641000BB279395F695879577956795B795F11175
:10642000F8CFFAF4BB0F11F460FF1BC06F5F7F4F12
:106430008F4F9F4F16C0882311F096E911C0772324
:1064400021F09EE8872F762F05C0662371F096E82D
:10645000862F70E060E02AF09A95660F771F881FFC
:10646000DAF7880F9695879597F90895990F0008A0
:10647000550FAA0BE0E8FEEF16161706E807F90716
:10648000C0F012161306E407F50798F0621B730BB1
:10649000840B950B39F40A2661F0232B242B252B32
:1064A00021F408950A2609F4A140A6958FEF811DD5
:1064B000811D08950E946D320C94DE320E94D0320C
:1064C00038F00E94D73220F0952311F00C94C73297
:1064D0000C94CD3211240C9412330E94EF3270F3DD
:1064E000959FC1F3950F50E0551F629FF001729F79
:1064F000BB27F00DB11D639FAA27F00DB11DAA1F88
:10650000649F6627B00DA11D661F829F2227B00DD4
:10651000A11D621F739FB00DA11D621F839FA00D5F
:10652000611D221F749F3327A00D611D231F849FAF
:10653000600D211D822F762F6A2F11249F57504006
:106540009AF0F1F088234AF0EE0FFF1FBB1F661F81
:10655000771F881F91505040A9F79E3F510580F04A
:106560000C94C7320C9412335F3FE4F3983ED4F39B
:10657000869577956795B795F795E7959F5FC1F7EE
:10658000FE2B880F911D9695879597F9089597F999
:106590009F6780E870E060E008959FEF80EC0895C9
:1065A00000240A94161617061806090608950024F2
:1065B0000A9412161306140605060895092E03946C
:1065C000000C11F4882352F0BB0F40F4BF2B11F4E0
:1065D00060FF04C06F5F7F4F8F4F9F4F089557FD3F
:1065E0009058440F551F59F05F3F71F04795880F41
:1065F00097FB991F61F09F3F79F0879508951216D8
:1066000013061406551FF2CF4695F1DF08C0161683
:1066100017061806991FF1CF869571056105089434
:106620000895E894BB2766277727CB0197F908954B
:10663000F999FECF92BD81BDF89A992780B508954A
:10664000262FF999FECF1FBA92BD81BD20BD0FB68E
:10665000F894FA9AF99A0FBE019608952F923F92F4
:106660004F925F926F927F928F929F92AF92BF9262
:10667000CF92DF92EF92FF920F931F93CF93DF930E
:10668000CDB7DEB7CA1BDB0B0FB6F894DEBF0FBE6B
:10669000CDBF09942A88398848885F846E847D84B8
:1066A0008C849B84AA84B984C884DF80EE80FD80BA
:1066B0000C811B81AA81B981CE0FD11D0FB6F89430
:1066C000DEBF0FBECDBFED010895A29FB001B39F05
:1066D000C001A39F700D811D1124911DB29F700DEB
:1066E000811D1124911D08955058BB27AA270E948F
:1066F0008C330C94DE320E94D03238F00E94D732B4
:1067000020F039F49F3F19F426F40C94CD320EF4A6
:10671000E095E7FB0C94C732E92F0E94EF3258F363
:10672000BA17620773078407950720F079F4A6F576
:106730000C9411330EF4E0950B2EBA2FA02D0B0103
:10674000B90190010C01CA01A0011124FF27591BB6
:1067500099F0593F50F4503E68F11A16F040A22FBC
:10676000232F342F4427585FF3CF4695379527952D
:10677000A795F0405395C9F77EF41F16BA0B620B2C
:10678000730B840BBAF09150A1F0FF0FBB1F661F73
:10679000771F881FC2F70EC0BA0F621F731F841FB6
:1067A00048F4879577956795B795F7959E3F08F0DC
:1067B000B0CF9395880F08F09927EE0F979587959E
:1067C00008950E94F5330C94DE320E94D73258F0BF
:1067D0000E94D03240F029F45F3F29F00C94C73278
:1067E00051110C9412330C94CD320E94EF3268F3A5
:1067F0009923B1F3552391F3951B550BBB27AA277A
:1068000062177307840738F09F5F5F4F220F331FB3
:10681000441FAA1FA9F335D00E2E3AF0E0E832D07B
:1068200091505040E695001CCAF72BD0FE2F29D07E
:10683000660F771F881FBB1F261737074807AB0750
:10684000B0E809F0BB0B802DBF01FF2793585F4FC5
:106850003AF09E3F510578F00C94C7320C941233F5
:106860005F3FE4F3983ED4F3869577956795B795A7
:10687000F7959F5FC9F7880F911D9695879597F9B2
:106880000895E1E0660F771F881FBB1F621773072B
:106890008407BA0720F0621B730B840BBA0BEE1F40
:1068A00088F7E09508950E945A346894B1110C94C9
:1068B000123308950E94F73288F09F5798F0B92F4D
:1068C0009927B751B0F0E1F0660F771F881F991F25
:1068D0001AF0BA95C9F714C0B13091F00E94113383
:1068E000B1E008950C941133672F782F8827B85F93
:1068F00039F0B93FCCF3869577956795B395D9F77D
:106900003EF490958095709561957F4F8F4F9F4F86
:1069100008950E94363208F48FEF08950E943632AF
:10692000880B990B0895A1E21A2EAA1BBB1BFD012F
:106930000DC0AA1FBB1FEE1FFF1FA217B307E4075E
:10694000F50720F0A21BB30BE40BF50B661F771FB6
:10695000881F991F1A9469F7609570958095909596
:106960009B01AC01BD01CF010895052E97FB1EF4DC
:1069700000940E94CC3457FD07D00E94933407FC4A
:1069800003D04EF40C94CC3450954095309521951D
:106990003F4F4F4F5F4F089590958095709561954B
:1069A0007F4F8F4F9F4F0895DF93CF931F930F9388
:1069B0009A9DF02D219FF00D8B9DF00D8A9DE02D6D
:1069C000F10D039FF00D029FE00DF11D4E9DE00DB6
:1069D000F11D5E9DF00D4F9DF00D7F936F93BF9263
:1069E000AF925F934F93D5010E9465338B01AC0149
:1069F000D7010E946533EB01E80FF91FD6010E9411
:106A000023352F913F91D6010E946533C60FD71FC2
:106A1000E81FF91FAF91BF910E9423352F913F913D
:106A20000E946533C60FD71FE81FF91FD6010E94C9
:106A30006533E60FF71F9801BE01CF010F911F913B
:106A4000CF91DF9108950E946533460F571FC81FED
:106A5000D91F08F43196089597FB57FF0C943C35E5
:106A60009F938F930E943C356E1B7F0BAF91BF911C
:106A70008A0B9B0B0895E894DF93CF93FC01DB0115
:106A80000E9465337F936F93E9019A01AC01BF9334
:106A9000AF933F932F93DF010E94653326F46C1B65
:106AA0007D0B820B930B9E01EB01FC010E942335B1
:106AB000AF91BF912F913F910E942335BE01CF012D
:106AC000F9012F913F91CF91DF910895689401C012
:106AD000E894F92FF12B12F00C949A35A0E0B0E075
:106AE000E4E7F5E30C943433092E059422F40E9474
:106AF000F635112392F4F0E80F26FFEFE094F094BE
:106B000000951095B094C094D094A194BF0ACF0A78
:106B1000DF0AEF0AFF0A0F0B1F0B0E94A53507FCC7
:106B20000E94F635CDB7DEB7ECE00C945033689494
:106B300001C0E8948F929F92CF93DF930E94A53576
:106B4000DF91CF919F908F90089588249924F4012C
:106B5000E401B0E49F93AA279A158B049C04ED05E9
:106B6000FE05CF05D007A10798F4AD2FDC2FCF2F5E
:106B7000FE2FE92D982C892E982F872F762F652FA1
:106B8000542F432F322F2227B85031F7BF9127C0FF
:106B90001B2EBF91BB27220F331F441F551F661F9B
:106BA000771F881F991F881C991CEE1FFF1FCC1F81
:106BB000DD1FAA1FBB1F8A149B04EC05FD05CE0533
:106BC000DF05A007B10748F08A189B08EC09FD090A
:106BD000CE09DF09A00BB10B21601A94E1F62EF467
:106BE0009401AF01BE01CD01000C08956095709530
:106BF0008095909530954095509521953F4F4F4FFA
:106C00005F4F6F4F7F4F8F4F9F4F0895002E08307B
:106C100090F0982F872F762F652F542F432F322FE8
:106C200022270850F4CF220F331F441F551F661F21
:106C3000771F881F991F0A95B2F7002D089597FDB9
:106C40001094002E083098F00850232F342F452F31
:106C5000562F672F782F892F912DF4CF1594979564
:106C600087957795679557954795379527950A9511
:106C7000AAF71124002D08952A0D3B1D4C1D5D1D02
:106C80006E1D7F1D801F911F08952A153B054C0521
:106C90005D056E057F058007910708950024A7FD17
:106CA00000942A17300540055005600570058005E1
:106CB00090050895EE0FFF1F0590F491E02D0994C3
:106CC0000F931F93CF93DF938230910510F482E0EE
:106CD00090E0E0914F07F091500730E020E0B0E005
:106CE000A0E0309799F42115310509F44AC0281B1A
:106CF000390B24303105D8F58A819B8161157105E6
:106D000089F1FB0193838283FE0111C0408151818F
:106D10000281138148175907E0F04817590799F481
:106D2000109761F012960C93129713961C9332965B
:106D3000CF01DF91CF911F910F91089500934F07DD
:106D400010935007F4CF2115310551F04217530726
:106D500038F0A901DB019A01BD01DF01F801C1CFC3
:106D6000EF01F9CF9093500780934F07CDCFFE01ED
:106D7000E20FF31F819391932250310939832883C5
:106D8000D7CF20914D0730914E07232B41F420910E
:106D90006E0130916F0130934E0720934D07209183
:106DA0006C0130916D012115310541F42DB73EB7CD
:106DB0004091700150917101241B350BE0914D07FA
:106DC000F0914E07E217F307A0F42E1B3F0B281794
:106DD000390778F0AC014E5F5F4F2417350748F054
:106DE0004E0F5F1F50934E0740934D078193919331
:106DF0009FCFF0E0E0E09CCFCF93DF930097E9F0E6
:106E0000FC01329713821282A0914F07B091500774
:106E1000ED0130E020E01097A1F420813181820F54
:106E2000931F20914D0730914E072817390709F01D
:106E300061C0F0934E07E0934D07DF91CF91089525
:106E4000EA01CE17DF07E8F54A815B819E01411513
:106E50005105B1F7E901FB83EA8349915991C40FC8
:106E6000D51FEC17FD0761F4808191810296840F94
:106E7000951FE90199838883828193819B838A830B
:106E8000F0E0E0E012968D919C9113970097B9F590
:106E90002D913C911197CD010296820F931F209165
:106EA0004D0730914E072817390739F6309751F5BD
:106EB0001092500710924F07B0934E07A0934D07C2
:106EC000BCCFD383C28340815181840F951FC817E3
:106ED000D90761F44E5F5F4F88819981480F591F30
:106EE000518340838A819B8193838283211531055D
:106EF00009F0B0CFF0935007E0934F079ECFFD010C
:106F0000DC01C0CF13821282D7CFB0E0A0E0EBE863
:106F1000F7E30C9430338C01009751F4CB010E94BD
:106F200060368C01C801CDB7DEB7E0E10C944C337C
:106F3000FC01E60FF71F9C0122503109E217F3070D
:106F400008F49DC0D901CD91DC911197C617D707E0
:106F500098F0C530D10530F3CE0104978617970716
:106F600008F3C61BD70B2297C193D1936D937C93E3
:106F7000CF010E94FC36D6CF5B01AC1ABD0A4C0192
:106F80008C0E9D1EA0914F07B0915007512C412CA3
:106F9000F12CE12C109731F580914D0790914E071F
:106FA0008815990509F05CC04616570608F058C0C8
:106FB00080916C0190916D01009741F48DB79EB75F
:106FC0004091700150917101841B950BE817F907EE
:106FD00008F055C0F0934E07E0934D07F901718317
:106FE0006083A0CF8D919C91119712966C9012970F
:106FF00013967C901397A815B90559F56C0142E0DA
:10700000C40ED11CCA14DB0420F1AC014A195B097F
:10701000DA011296159780F0628273825183408361
:10702000D9016D937C93E114F10471F0D7011396AB
:10703000FC93EE93129776CF22968C0F9D1FF90149
:1070400091838083F301EFCFF0935007E0934F07D4
:1070500069CF4816590608F42C017D01D3019ACF57
:10706000CB010E9460367C01009749F0AE01B80167
:107070000E944238C8010E94FC36870153CF10E0BD
:1070800000E050CFFB01DC0102C001900D924150A5
:107090005040D8F70895FB01DC018D9101908019D3
:1070A0000110D9F3990B0895FB01DC0101900D92B9
:1070B0000020E1F70895FB01DC014150504030F021
:1070C0008D910190801919F40020B9F7881B990B54
:1070D000089510E0C2E6D0E004C0FE010E945A36D6
:0C70E0002196C336D107C9F7F894FFCF02
:1070EC00011F1115111D1D111F1F11151115151142
:1070FC001F1F111D1D1D1D1D1F1F111711151511F2
:10710C001F1F1117111D1D111F1F1515111D1D1DE1
:10711C001F1F111D111D1D111F020701D0B13700BA
:10712C00960032000500E1000040787D018C5C0384
:10713C0000A03B4C000F0401204E000040420F0009
:10714C005073370000046BF414000000000051076A
:10715C0080000000400014005400000204000300F2
:10716C0001100302000003020100060004000605E2
:10717C000020060504000000000037059704C40435
:10718C008405F504D304E7040000000076074907E2
:10719C00F60726073C013607270700000000C10947
:1071AC009704F60788046E616E00696E66006F7650
:1071BC006600494600464130303030303031303096
:1071CC0030303B00464130303033303030303030AE
:1071DC00303B003031003034003035003036003078
:1071EC00390030330030370054583B00535752208D
:1071FC002020202020503D305720202020200053DC
:10720C0057523D0020503D0057202020002D0041BA
:10721C006D7065722E203D20002041005A5A534D4E
:10722C0030005A5A5041004F666620004C6F772050
:10723C00004D6564200048696768004642004F00B5
:10724C005A5A53443B004552524F522053544550C6
:10725C003E32354B487A003F005541525400204293
:10726C006175640020202020506F77657253445262
:10727C002020202000202020444953434F4E4E45CF
:10728C004354202020003032005344522053696E66
:10729C0074657A205554334D4B00536F66742E4DE4
:1072AC0069636B795F76362E33410052582020008B
:1072BC00545820200052583B0030303030003031D0
:1072CC003131005A5A53553B0042553B0031363050
:1072DC000042443B0052454320005A5A51533B0054
:1072EC005A5A5041303B005A5A5041313B005A5A7D
:1072FC005041323B005A5A5041333B004641005AF0
:10730C005A4D4430323B00467243616C0020487A3F
:10731C002000434C4B302000537465703D00436F8C
:10732C0072722E504C4C5F464958454400204D48D3
:10733C007A00436F7272465245512E20515541527C
:10734C00545A0020487A00434F4D20504F5254203D
:10735C0052532D32333200426175643A200045722B
:10736C00617365205369646542616E64200020532B
:10737C00656320004F6666202000465245512E451D
:10738C00722E5369646542616E640044656C617968
:10739C005458200044656C61795458204F6666003F
:1073AC0044656C61795258200044656C617952587F
:1073BC00204F6666004175746F20415454202B0099
:1073CC00644220004175746F2041545420204F6654
:1073DC0066005A5A4D4400205374657020002048B2
:1073EC007A202020200056666F0046423B005A5AF5
:1073FC00534D303B00FFFFFFFFFFFFFFFF0700FF78
:10740C00FFFFFFFFFFFF062020202020202000FF91
:10741C00FFFFFFFFFF05202020202020202000FF61
:10742C00FFFFFFFF0420202020202020202000FF31
:10743C00FFFFFF032020202020202020202000FF01
:10744C00FFFF02202020202020202020202000FFD1
:10745C00FF0120202020202020202020202000FFA1
:10746C00FF2020202020202020202020202000FF72
:10747C002020202020202020202020202020002020
:10748C002020202020202020202020202020005AD6
:10749C005A50413B004C6F6164005A5A51523B00A8
:1074AC0038300034300033300032300031370031A6
:1074BC00350031320031300055503B00444E3B001A
:00000001FF
